:020000040800F2
:1050000070340020D55000085DA70008DD9C000822
:105010000000000000000000000000000000000090
:10502000000000000000000000000000D1B50008F2
:105030000000000000000000D9AC0008ADBC000872
:10504000E7500008E7500008E7500008E750000864
:10505000E7500008D5660008E7500008E56600083C
:1050600000000000E7500008E7500008E750000883
:10507000E7500008E59F0008E7500008E7500008E7
:10508000E7500008E7500008E75000080000000063
:10509000E7500008E7500008E7500008E750000814
:1050A000E7500008E7500008E750000899CA0008D8
:1050B000A9CA000825A100080000000000000000A7
:1050C0000348854600F040FD004800475DE50008C4
:1050D000703400200448804704480047FEE7FEE79C
:1050E000FEE7FEE7FEE7FEE76DBD0008C1500008E1
:1050F00030B50B46014600202022012409E00D4670
:10510000D5409D4205D31D469540491B25469540F7
:1051100040191546521E002DF1DC30BDF0B51FB40C
:105120000646002082B005464024019100901BE015
:10513000019922460F46304600F0EAFB049A059B8F
:10514000801A994110D310461946224600F0D0FB30
:10515000361A8F410197224601200021009F00F05E
:10516000C7FB38184D4100902046641E0028DFDC44
:10517000019B00982946324607B0F0BD03460B4319
:105180009B0703D009E008C9121F08C0042AFAD2FD
:1051900003E00B780370401C491C521EF9D2704783
:1051A000D2B201E00270401C491EFBD270470022BF
:1051B000F6E710B513460A4604461946FFF7F0FF16
:1051C000204610BD30B505462A460B4610781C789F
:1051D000521C5B1C002801D0A042F7D0002C03D049
:1051E000002802D06D1CEFE7284630BD421C017834
:1051F000401C0029FBD1801A704730B504460020BE
:10520000034600E05B1C934203D2E05CCD5C401B94
:10521000F8D030BD70B5064607F06CFF046805464F
:105220000A220021304600F097FB2C6070BDF8B5D3
:1052300002464A40D40F42004B0052085B089A4293
:1052400002D20246084611464A0023D0C30D4A0046
:10525000DDB2120EAD1A202D35DA49020126490AB7
:10526000F6058A19002C00D0524220214F1B11460E
:10527000B9402A411018C20D9A4221D0002C17D0F3
:10528000012D08DCDA05801AD20F8019D207DBB2B3
:1052900000F0A2FBF8BDDA05801A012340001B06CE
:1052A000C01880185A428018CA0F1043490007E0FE
:1052B0004908C2071143DA05801A8019400880188E
:1052C00000F082FBF8BD61000122511A001BF7E7D4
:1052D0000122D2075140AAE70122D2075040A6E797
:1052E000024670B54A40D30FDB0740002DD04A007C
:1052F0002AD0010E140E000212020919400A520AA5
:105300008418E50104465443000A120A2E0450434F
:10531000A4194219200CC543AA18120C0125AD038B
:10532000521C521912047F39240400D0521C10431D
:1053300001D44000491EC2B20C06C0092018401C0E
:105340004008802A02D003E0002070BD40084000E1
:10535000002900DA0020184370BD70B502464A40AB
:10536000D50F40004A00ED0740085208002814D02D
:10537000002A12D0C40DD30D41020120C0055202F3
:10538000490A520AE41A091812187D34914201D3CD
:10539000641C00E04900002C01DA002070BD0023ED
:1053A000914201D3891A0343400849000028F7D1EC
:1053B00000290AD0914202D10121C90705E091429A
:1053C00001D2012101E00121C943E005C0184019C3
:1053D00000F0FAFA70BD420005D04200120E5242AF
:1053E0008A4201DB00207047C90508187047000099
:1053F000F0B507460846584087B0C00F04904800F3
:105400000E46590040084908BC1A884105D2384662
:1054100031461E4617460B460246580040081043C8
:105420004CD0300D039040055900400D490D0590BA
:10543000401A0290402872DA18030121000B090576
:105440000843019004980092002805D00199524227
:105450000020884100920190029840210A1A019987
:10546000009800F045FA05460C466B4607CB00F065
:1054700060FAC0197141039A0E0D0023D7175640E8
:105480001A467A40164344D0049A002A2DD0029A34
:10549000012A039A15DC1205C01A9141012636052E
:1054A000001C7141D20F059ED20700930192029613
:1054B0002A46234600F0D6FA07B0F0BD38463146FA
:1054C000FAE71605224A0F46B218C01AB741012161
:1054D0000905001C4F4100187F41114618187941F9
:1054E000E20F10436D19644113E0E2076D081543A4
:1054F0006408C2071443039A01261205C01A914199
:105500003605001C7141CE07400830434908C018D9
:1055100051412A46234600F098FACDE7FFE7049868
:1055200001224000C117121A00238B410498314612
:10553000C417381AA141EEE730B40124E4076340F0
:1055400030BC55E730B40124E407614030BC4FE77C
:105550000000E0FFF0B51FB488B00B990998002453
:1055600048400999C00F490049080991C0070B99A3
:105570000090490049080B9109990898A6460843EC
:105580001CD00B990A98084318D0099801244000B0
:10559000420D4800410D099824050003000B2043EB
:1055A00009900B980003000B20430B9050181C49E6
:1055B0004018002201901446104605E000200146E4
:1055C0000DB0F0BD032801DA034600E003239C463A
:1055D000C11A0AAE0AE05F0008ADED5B4F00F75B51
:1055E0007D430027AA187C41491C5B1E6145F2DD02
:1055F000410004AB5A522104120C0A43240C401CF3
:105600000828DFDB01980290009970460191009014
:10561000059B049A0799069800F024FAD0E7000049
:105620000DFCFFFFF0B50C465C4085B0E40FE407CD
:1056300003944C0000266408590094464908024629
:105640000296224321D062460A431ED06200570DC3
:105650004A000E032303550D012402462C4924055C
:10566000781B1B0B360B40182343264361460090E2
:105670001C46501AB44103D30098401C009002E02D
:10568000921800985B41002803DA0020014605B01B
:10569000F0BD0020012109050746864611E0644659
:1056A0001D46141BB54106D36546521BB3417446D3
:1056B00007430C43A646CD074008490828439218E3
:1056C0005B4105460D43EAD11046184313D06046AE
:1056D000194650407140084306D06046101AB34145
:1056E00006D20122002306E000220123DB0702E0AC
:1056F0000122D2435310009874460105381C6141C1
:10570000029C039D0019694100F09FF9BFE700006A
:10571000FD03000070B54B005B0803430BD04B004A
:105720005C0D002633466542B341D417AD1AA34140
:1057300002DB0020014670BD12053018514170BDDA
:1057400010B500229623114600F046F910BD000066
:105750000EB5C217C10F5040CA0740180021054BB3
:105760000293019200910A460B4600F07BF903B0C8
:1057700000BD0000330400000EB505490291002170
:1057800000910A460B46019100F06CF903B000BD90
:1057900033040000410040020122400AD205090EF4
:1057A00080187F2901DA00207047962903DC9622B1
:1057B000511AC840704796398840704770B5CD0F70
:1057C0004A0009030123090B1B0519430B4BED0785
:1057D0000024520D9A4201DA002070BD074B343389
:1057E0009A4203DC9A1A00F093F802E00449511837
:1057F00088402C43F1D0404270BD0000FF03000000
:10580000CDFBFFFF4A0009030123090B1B051943C8
:10581000094B10B5520D9A4201DA002010BD064B1B
:1058200034339A4203DC9A1A00F072F810BD03492F
:105830005118884010BD0000FF030000CDFBFFFFA2
:10584000C20FD207400040080BD0C10D0723DB0177
:10585000C91840020905400A1143C2084007114314
:10586000704700200146704710B5002904DB012471
:10587000E40740428C412146002B04DB1C460123F7
:10588000DB075242A3418B4200D1824210BD00008F
:1058900010B5002904DB0124E40740428C41214675
:1058A000002B04DB1C460123DB075242A341994233
:1058B00000D1904210BD0000CB0FDB07490010B5AE
:1058C000490802460A4307D00A0D07240903E401E8
:1058D000090B121B002A01DC002010BDC900440F77
:1058E0000C43C100E018D205801800F06DF810BD1F
:1058F00010B5202A04DB0146203A9140002010BD5B
:10590000914020239C1A0346E3401943904010BD68
:1059100010B5202A04DB0846203AD040002110BDF3
:105920000B46D340D0402024A21A91400843194688
:1059300010BD10B5202A06DBCB170846203A1041CF
:10594000C1170B4306E00B461341D0402024A21A96
:1059500091400843194610BDF7B5009C0F4600263C
:105960002578641C002D05D000F000F90068405D2A
:10597000C007F5D12B2D02D02D2D18D0641E39462D
:105980002046029A00F0F6F8002F04D03968A142B0
:1059900001D1009939607105022400290BDA4042D7
:1059A000002803DD07F0A6FB0460A007FEBD012070
:1059B00080020643E3E70028F8DA07F09BFB046067
:1059C0000048FEBDFFFFFF7F002904DA401C4900AC
:1059D00001D140084000704770B40024050C05D187
:1059E0001024000402D1002921D01124050E01D178
:1059F00000020834050F01D10001241D850F01D1DB
:105A00008000A41C002801DB4000641C002908D091
:105A100020252E1B0D46F540A14000D00121294331
:105A2000084301061B1B000ADB1D02D5002070BCC9
:105A30007047DB05181880180029F8DA401C490067
:105A4000F5D170BC40084000704710B5002B08DA53
:105A50000024401C614192185B411A4301D1400867
:105A6000400010BDF0B51FB482B005460C0003D055
:105A7000084607F0E5FA02E007F0E2FA20300246B5
:105A8000009021462846FFF733FF049B059A044601
:105A90000F4618431143084314D0184610431BD037
:105AA000009840210A1A18460599FFF731FF05466C
:105AB0000E46009A05990498FFF71AFF084305D08F
:105AC000012004E02046394607B0F0BD0020C11790
:105AD00005430E432C43374300990E986305401A43
:105AE0007905E40A00220C43FD0A0A3002D50020A1
:105AF0000146E9E70105101969410C9C0D9D00194B
:105B00006941FFF7A2FFDFE74A0009030123090B00
:105B10001B0519430A4B10B5520D9A4202DA0020B8
:105B2000014610BD064B34339A4203DC9A1AFFF744
:105B3000EFFE10BD034BD218FFF7DAFE10BD0000D8
:105B4000FF030000CDFBFFFF064C0125064E05E0DC
:105B5000E36807CC2B430C3C98471034B442F7D38E
:105B6000FFF7B2FAC0ED0008E0ED0008004870470A
:105B700020EC0008F7B582B0029C00272078641C56
:105B800015460197302802D0002D15D015E0207859
:105B90000127641C782804D0582802D0002D09D091
:105BA0000BE0002D01D0102D07D100271025207803
:105BB000641C02E0082500E00A250026009610E09B
:105BC0000099012769430818020C294680B27143E5
:105BD00000908E183804864201D30120019020786D
:105BE000641C294600F019F80028E9DA0398002817
:105BF00005D0002F01D0641E00E0029C04600198D3
:105C0000002806D007F076FA02210160C81E05B010
:105C1000F0BD009930040843F9E73A2800D2303843
:105C2000202302469A43412A01D31046373888423E
:105C300001D30020C043704770B58C180578401C14
:105C40006B075B0F01D10378401C2A1106D1027843
:105C5000401C03E006780E70401C491C5B1EF9D105
:105C60002B0705D40023521E0DD40B70491CFAE7F4
:105C70000378401CCB1A921C03E01D780D70491C60
:105C80005B1C521EF9D5A142D8D3002070BD70B55F
:105C9000044620688168490727D58168102549078F
:105CA000002905DA8168890702D481682943816067
:105CB00001F020FD064620688068400715D501F0F8
:105CC00019FD801B0A280CD920688068400708D578
:105CD000606D28436065A06D01210843A065012027
:105CE00070BD206880684007E9D4002070BD0000C6
:105CF00038B50446094808490068FFF7F9F96043D8
:105D000000900098002805D00098401E0090009850
:105D10000028F9D138BD000040420F007C0200206D
:105D2000F8B50446206881688907890F012934D1B4
:105D30000168C90731D0816805221140102501266C
:105D4000012907D0606D28436065A06D3043A065D0
:105D50000120F8BD8168022211438160216803207F
:105D6000086001F0C7FC074620688068C00714D0AF
:105D700001F0C0FCC01B0A280BD920688068C0074E
:105D800007D0606D28436065A06D3043A065012099
:105D9000F8BD20688068C007EAD10020F8BD000087
:105DA000F8B50446206881688907890F012902D166
:105DB0000168C90733D181681A4A102611400125AC
:105DC000002907D0606D30436065A06D2843A06551
:105DD0000120F8BD8168294381600120FFF788FF19
:105DE00001F088FC074620680068C043C00716D051
:105DF00001F080FCC01B0A280CD920680068C04351
:105E0000C00707D0606D30436065A06D2843A06572
:105E10000120F8BD20680068C043C007E8D1002019
:105E2000F8BD00001700008010B50E4801F05CFAC4
:105E300000F00AFA05F070FD00F04EFD0A480B492B
:105E4000C08C08600A4C0020E06000F015F809489A
:105E500000F0B6FE00F08CF8207004F0A3F90020EA
:105E600010BD0000B80B00002C0800202C00002002
:105E70003C000020CD68000810B5012008F058FC57
:105E80000A4C1328A0700AD0E01C04F05FF8E078F8
:105E9000A070332806D006490020C88710BD08F03E
:105EA0007FFC10BD04F024F810BD00002802002083
:105EB000EC07002010B500F003F8002010BD000032
:105EC00070B50524FF22240701322146012004F089
:105ED0001DFF1749002006F0E3FE1649022006F0D8
:105EE000DFFE1549012006F0DBFE144D012292036E
:105EF0002946002004F080F904222946012004F0FC
:105F00007BF9012212032946022004F075F91022C0
:105F10002146002000F0F4FD0021094800F0DCF8E3
:105F20000122D2022146012000F070F8002070BD4D
:105F300044060020CC060020BC05002000040050D0
:105F4000AC07002010B50024084801F0FBF8611EE2
:105F5000064801F08FF8002803D1044800F064FFE0
:105F60000446024801F01EF9204610BD300500200D
:105F700070B5002400F026F80D4E0546B04215DB42
:105F800000200C4A0C4B0146FFF782FC01D264242E
:105F90000CE031462846FFF79BF90849FFF7DDF989
:105FA0000749FFF79DF9FFF7F5FB0446204670BD52
:105FB00033335340CDCCCCCCCCCC10406666663F5E
:105FC0000000C84210B500F017F8642001F08CF909
:105FD000FFF7B8FF00F028F8044600F003F8204669
:105FE00010BD000010B5034801228189806801F0CE
:105FF0007AFB10BDEC16002010B503480022818901
:10600000806801F070FB10BDEC160020022802D35E
:106010000020C0437047C3000248C1501818828056
:1060200000207047EC16002010B5FFF7A5FB0022FA
:10603000064BFFF7F7FA064A064BFFF78BFAFFF716
:106040003BFC0121FFF7C7F910BD000000FEAF4087
:106050006666666666660A4010B50D4C00232046EB
:1060600000686168026800290BD004290BD0082958
:106070000BD0136402F04CFD206802F0BBFB002043
:1060800010BD5363F6E79363F4E7D363F2E70000D0
:106090005401002010B50F4C206802F07BFB03CCAC
:1060A000083C02F0EBFC61683C20002908D0042980
:1060B0000AD00829216809680AD00864002010BDA8
:1060C000216809684863F9E7216809688863F5E78A
:1060D000C863F3E754010020014A03C2002070475F
:1060E00054010020F0B5454D89B0002444486700B4
:1060F0000246015D5C32D153032909D04049A20018
:10610000404830398850641C0B2CEFDB09B0F0BDDF
:10611000022101553A48A600F8308059FFF718FBD4
:10612000394A3A4BFFF716FAFFF7C6FB686502904B
:106130003348A96DCC308059401AFFF71DFB6967C1
:106140002867059106902E482D49A030743180595A
:106150008959401AFFF710FBE967A867049003917B
:106160007F20C0050299FFF7B3F8FFF769FB039B97
:10617000049AFFF7EFF9059B069AFFF7E3F900226F
:10618000D243FFF7C7FA224A224BFFF7E3F91B4A33
:10619000214B803203C213221206FFF7DBF9E966B6
:1061A00000221E4BA866FFF773FB22D200221C4B75
:1061B000E96EA86EFFF758FB1BD21A48C05FFFF7C5
:1061C000C7FA039107460022174BE96EA86EFFF746
:1061D000C1F93A46039BFFF70BF9FFF7EFFA0849BD
:1061E00030398851287803288DD1E87A401CE8722C
:1061F00089E7034903483039885184E7A800002023
:10620000100F0020FFFF0100143BB1133BB103BE90
:10621000FA48CE3B1835B13D19DDB141000024C02C
:1062200000408F40341000200000594010B500237A
:106230001A4603E0845CE3189BB2521C8A42F9D3ED
:10624000D84380B210BD000000B587B00121684678
:106250004170022101700D480190C8010290800038
:106260000490402005906946002006F065FC074830
:106270000749203801610749C16107498161074920
:106280004161074803F072F907B000BDEC1500202A
:10629000B1620008A5620008E1620008EF62000830
:1062A0004C10002010B50146002006F005FC10BD82
:1062B0000FB400B5FFB082B0012183AB490268463C
:1062C000829A06F0A7FE6846FEF790FF02466946EE
:1062D000002006F049FD7FB002B008BC04B01847AA
:1062E00001B501226946002006F03EFD08BD10B54B
:1062F0000446FEF77BFF02462146002006F034FDEF
:1063000010BD30B4446C1C252C400125A540046C04
:106310006560046863608368102B05D0036899602A
:106320000068C26030BC704703689A600068C16052
:1063300030BC704708B503E06846007806F0C2FD3F
:106340006946002006F0B8FB0028F5D008BD000023
:10635000F8B50A2007F0B9FF002007F0D1FFA64CDE
:1063600000266670A548E0646676607C0C2801D340
:106370000B2060740A212171A148A670A14D0078FC
:106380002871A14A6079127840001043A27D9200E2
:106390001043227E52011043E871E06AE870020A5D
:1063A0002A72401CE062A9742846142297491330CF
:1063B000FEF7E4FE954928462C2227306031FEF78F
:1063C000DDFE9249284616225330EC31FEF7D6FE08
:1063D0008F480021415E002903D08E4A128A51184D
:1063E00001808849027850314A76407888761A20B0
:1063F000687289480078A872A07F287308467E4991
:10640000633820310A780275497841756D20002281
:106410007C4908F045F820790021C0001D3008F0C3
:1064200051F806F0D7FD022007F0A0FF0026EE711C
:10643000A674A67301202074E673784801F0B2FABE
:10644000A0840546A6702079FFF796F9744A754B2B
:10645000FFF780F807F094FB0022734BFEF7C8FFAC
:10646000FFF7D0F90006C10C481980B20121C90319
:10647000E084884201D3401AE0846C48A063E0784D
:10648000401CE070654801F08DFA6084684E53E06E
:10649000624801F087FA6084664D0AE05F4801F0C7
:1064A00081FA80B26084E18C884202D389198842E3
:1064B00006D300210F2007F075FE28422063EDD09F
:1064C000206B411C22D0400436D58122D20100210C
:1064D0000F2007F0BAFF0021102007F063FE4106ED
:1064E0004A48490E0022A438A16407F0ABFE07F029
:1064F0006DFE2065002007F003FF002007F0BBFEC3
:106500004248A438417A172902D008E006F0E4FD99
:1065100002224949401DFEF770FE002836D02A4667
:1065200000210F2007F091FF2079A178401C8142C3
:1065300002D0002007F09FFE618CE08C8142A7D33F
:1065400080198142A4D807F04BFDFFF7CBFD3B4BF0
:106550002E4A0021184660328D005559854203D2DB
:1065600028462A4D4E00AF5B491CC9B20B29F3D314
:10657000984204D0278400206073012020702D4AA7
:10658000002180320F2007F060FFF8BD07F0D3FF35
:10659000E165A06507F0BCFF616603462066A07850
:1065A0001A4A401CC0B2A070AB3A157A69460D7009
:1065B000527A4A7005464200144809888152134AAB
:1065C00082380090863A2846111F05F065F80F4A78
:1065D0000321903251551046A9003038405860636D
:1065E000A06C2628A8D1114668005C3141180748E4
:1065F0008C38008808809FE7A80000203F420F00E9
:106600003C000020280D002060000020800E0020AB
:106610008A0000202C080020780000208C05002033
:106620009A9999999999E13F00000840A086010044
:10663000983A000000D0272468000020FFFF0100E6
:106640001449012048720A4602205E32507203202B
:106650003C3A507204200E3A50720F480D4B0078AD
:10666000087022310870203108770C495A1C0878CC
:1066700058714978997123331871597120331877FB
:106680005977107551751A461E321075517510766E
:1066900051767047B40C00206E0000206800002086
:1066A00010B504F06DFF202005F0D2FA012007F0AC
:1066B000BFFC002005F0CCFA044807F057FB044863
:1066C00007F014FE002007F049FE10BD94000020E2
:1066D0008380000010B5012000F038FF022000F098
:1066E00035FF10BD10B5202000F030FF802000F0F5
:1066F0002DFF10BD10B4084900234B6107494A68BB
:106700004C1522434A604A68082422434A60C00963
:10671000C001036010BC7047542D002000200240CF
:106720007FB500250C460646039500F05BFEE009A8
:10673000029003A901960095684600F0E7FD002845
:1067400004D000F023FE002004B070BD00F01EFE57
:106750000120F9E710B5002302E0C45CCC545B1CB7
:106760009342FAD310BD000010B40020204A916972
:10677000CB05204904D54869022318434861901588
:1067800093699B0505D54B69012423434B61630243
:10679000184393695B0505D54B69082423434B6176
:1067A000E301184393691B0505D54B690424234372
:1067B0004B616302184393699B0405D54B69102410
:1067C00023434B616302184393699B0304D54C69CF
:1067D00020231C434C6118439369DB0305D54B69A7
:1067E000402423434B61A1020843906110BC7047D1
:1067F00000200240542D002070B5044600F07AFFBE
:106800000546194EB069C0070DD0601C08D0002C99
:1068100004D000F06FFF401BA04201D9032070BDDF
:10682000B069C007F1D1B069800701D50220B0611D
:10683000B069C00511D4B06980050ED4B0694005B7
:106840000BD4B069000508D4B069800405D4B069E0
:10685000800302D4B069C00303D5FFF785FF012090
:1068600070BD002070BD000000200240F8B5174642
:10687000002605460C4600F0B5FD09E02946022039
:10688000226800F091FD002804D1241D2D1D361D25
:10689000BE42F3D300F07AFDBE4201D20020F8BD23
:1068A0000120F8BD10B5084902460020054B0979C2
:1068B00005E044001C5B944203D0401CC0B28842F7
:1068C000F7D310BD800E0020A8000020014902204F
:1068D000887170473C00002000B587B001206946F0
:1068E0004870022008700C490191410202910B4945
:1068F00003910521490204910590694606F01CF9AF
:106900008821074802F0E6FF052001221021000738
:1069100000F0E9FE07B000BDFC160020FC1A0020C4
:106920000C250020F0B593B00E460546282108A896
:10693000FEF73DFC03AA00922846314601AB4DA26A
:1069400002F0F9FF0027FF4302281AD104990398A7
:1069500002F0E1FFC2B201980178012003E0019B3F
:106960001B5C5940401C029B8342F8D8914208D1DD
:10697000002406AB42A23146284602F0DCFF0F2875
:1069800002D0384613B0F0BDA819801E04704470C0
:1069900047482B4602784748418804920291039465
:1069A000059445498088097801910090FF2143A210
:1069B0000131494803F0B2F8074680214748FEF705
:1069C000F6FB3A4644494548FEF7D8FB434DF9B239
:1069D000083DA9700698424E0078302825D03E48E0
:1069E00002F0B4FD6868002842D03EA002F08EFD9F
:1069F0006878002803D0FF2030606C7002E001202E
:106A0000346068703C483B4D3C4F01682B683268ED
:106A1000386804F01BFE642000F066FC34603648E1
:106A2000224601682B68386820E039462A4802F07F
:106A30008DFD6878002804D0FF20000230606C7063
:106A400002E00120346068702A4D2B4F2B482B68E0
:106A500032683968006804F0F9FD642000F044FCF5
:106A60003460264822462B683968006804F0EEFD41
:106A7000002087E72425702A25700D0A00000000F9
:106A800024252A2C252A2C252A2C252A2C252A2C7B
:106A9000252A2C25702C252A2C252A2C252A2C2524
:106AA0002A2C252A2C252A2C252A2C252A2A0000A6
:106AB00041000020EC0700203C00002025732C251D
:106AC000582C253032782C25782C25642C25782CD0
:106AD0002564250D0A00000094250020680100208F
:106AE000200000204C4F524120464146414641463D
:106AF000410D0A001C000020240000202800002076
:106B0000C3000248C150181882807047FC2400203E
:106B100008B500206946087003E06846007800F078
:106B200013F86946022005F0C7FF0028F5D008BD1C
:106B300001490020087070476001002001490120D0
:106B4000087070476001002070B51A4D00262C4671
:106B50002B78611C8034002B08D022465268022B0F
:106B60000CD0032B09D10A2813D021E0242804D10A
:106B700002222A7070540120606070BD5054616818
:106B8000491C61607E2913D20D28F6D1032028709C
:106B900070BD50546068401C6060465406A1681C7B
:106BA000FEF710FB002803D0681C6168FFF7BAFEEF
:106BB0002E7070BD0C2500204747412C00000000BE
:106BC00001494860704700006001002070B53B49F2
:106BD0003B4A00208300401CC0B2D1500C28F9D39E
:106BE000394938480A7802754978417537490A7831
:106BF00002764978417633491520133148720A20CC
:106C000007F063FB7D20400107F07AFB2D4900224D
:106C100013310C2007F044FC00210C2007F052FC3B
:106C200006F0D8F9022007F0A1FB274D284C203DA3
:106C300000210F2007F0B6FA20422863F8D0286B15
:106C4000411C38D0400435D58122D20100210F20CB
:106C500007F0FBFB0021102007F0A4FA41061948B9
:106C6000490E0022C73007F0EDFA164CC734607A9F
:106C700015281FD102221549601DFEF7BEFA002813
:106C800018D11148A67C2E710422611C2430FEF715
:106C900075FA21461331084672000C469130FEF712
:106CA0006DFA28792146420005484838FEF766FA11
:106CB0000320287070BD06F00FFA0000FFFF0100EE
:106CC000E00E0020150D0020C80000206800002004
:106CD00000D02724F8B50C4605464035297C01290B
:106CE0000DD00121297401688A68520709D5416DC8
:106CF000202211434165002028740120F8BD0220A4
:106D0000F8BD194B6268D8054710184E9A4215D045
:106D10008A6A23685B035B0B1A438A622168490312
:106D200005D5B1680143B1600A20FEF7E1FF206894
:106D3000800315D5B0683843B06011E08A6A2368D3
:106D40005B035B0B9A438A622168490302D5B168F1
:106D50008143B1602068800302D5B068B843B06059
:106D600000202874F8BD0000011000000027014039
:106D700070B50446002C0AD0606D0221084360659E
:106D80002046FEF784FF0546280002D009E00120D6
:106D900070BD2046FEF7C4FF0546012D01D001203D
:106DA00060650026012D32D0206841681A4A1140E2
:106DB00041602168D0430860206881680122120781
:106DC000914381602068C168144A1140C160206805
:106DD0000169134A1140016120684169C908C9006D
:106DE00041612068016A0F4A1140016220688030C9
:106DF000416BC909C901416320688030416BC909F1
:106E0000C9014163204600F0F9F8A6656665403483
:106E10002674284670BD000060F7FFFF00023E8325
:106E200002FCFF3F00F000F00068006C70470000BB
:106E300070B50446002C06D0606D2646002540360D
:106E4000002802D006E0012070BDA56535742046FB
:106E500000F0E8F8606DC00603D420688168490737
:106E600006D5606D1021084360653574012070BD42
:106E7000616DFF22013291430222114361658168F5
:106E80005C4A8907890F012902D10168C9072BD102
:106E9000032361689B07994205D05B42994202D067
:106EA0005B00994209D10169890089080161206864
:106EB00001696368194301610CE00169890089086F
:106EC000016190680F21890488439060906861682F
:106ED000084390602068C16818239943C160206806
:106EE000C168A3681943C1609068012149068843BD
:106EF00090609068A18E4906084390602068816880
:106F0000C90004D4816801221207114381602068FE
:106F1000C168394A1140C1602069E268022825D061
:106F200000200243204620300178037B49035B00A8
:106F300019430A43216B0A43A16989030A43E169A2
:106F4000C9030A432168CB681A43CA60616A0A46CA
:106F5000FF3AC23A05D0A26A11432268D3681943A6
:106F6000D16042780121012A02D00BE00420D8E749
:106F70000078002823D0606D202210436065A06D4A
:106F80000843A065E06B012820D020680169C9078B
:106F900003D0016949084900016120684169C908B5
:106FA000C900416120684169A26B11434161A56537
:106FB000606D80088000401C6065002070BD206806
:106FC000C26801231B041A43C260DBE72068026920
:106FD000FF239B009A43026120680269236CA66C20
:106FE0001A43636C33431A430261206802690A43FF
:106FF0000261D2E7002701401902FEFF10B50068C8
:107000000649884209D10648416B421591434163C4
:1070100005200221000700F015FA10BD00240140F0
:107020000010024010B586B0044614216846FEF7F1
:10703000BEF80E492068884216D10D48416B4215B2
:1070400011434163C16A01221143C162C06A6946AA
:107050001040059002200090032001900020029033
:107060000520000700F07EFA06B010BD00240140A4
:1070700000100240F8B504460E46274660694037C6
:1070800008280BD02068C068C00709D0606D202197
:1070900008436065002038740120F8BD082500E031
:1070A0000C2500F027FB009020680068284219D1C9
:1070B000701C13D0002E05D000F01CFB0099401A64
:1070C000B0420BD920680068284207D1606D0421C6
:1070D00008436065002038740320F8BD206800680C
:1070E0002842E5D0606D01214902084360652068AF
:1070F000C16809058A0F0C21002A1BD12022125DCC
:10710000002A17D10268120714D58268012352079A
:10711000002A08DB42688A434260606D1A0290438D
:107120001843606506E0606D202210436065A06D25
:107130001843A065A069002801D1206801600020E3
:10714000F8BD000070B50446002021688968490731
:1071500023D425464035297C01291CD001212974DE
:10716000E169012902D02046FEF71AFE002811D15C
:10717000616D0B4A1140FF2201321143616500210C
:10718000A165297422681C21116021688A68042382
:107190001A438A6070BD022070BD022070BD0000DD
:1071A000FEF1FFFF70B5044625464035287C0128D6
:1071B00007D001262E742046FEF769FD002802D074
:1071C0000CE0022070BD2046FEF7AAFD002805D184
:1071D000616DFF22013291433143616500212974C1
:1071E00070BD30B4014620314A790023022A05D00F
:1071F0000422C2630B7130BC01207047026814681E
:107200000E25AC43146002681468640864001460BE
:10721000446C1C22144001252A46006CA2404260A6
:107220004D710B7130BC1846704770B50024014693
:1072300020314A79022A03D00421C163012418E0D5
:10724000026813680E25AB431360026813685B087D
:107250005B001360436C1C22134001252A469A40B0
:10726000036C5A604D7100220A71816B002900D0B5
:107270008847204670BDF8B504468C460025204658
:1072800020300179012909D00126067147790021B2
:10729000012F05D0017102252846F8BD0220F8BD56
:1072A00002274771E16320680168490849000160CD
:1072B00061462046FFF725F8206B002805D020689E
:1072C00001680E221143016009E020680168042270
:1072D00091430160206801680A221143016020681F
:1072E000016831430160D7E770B5044600F002FA47
:1072F0000546601C02D004480078241800F0FAF912
:10730000401BA042FAD370BD70020020F8B50546BC
:107310000E461B4F387C012808D0012038741948CC
:10732000FFF76AFA0146080002D025E00220F8BD06
:107330000020C04330606C68A868C0010019A042FA
:107340001AD92046FFF7D6F90E48FFF755FA01463D
:107350000D48426808239A434260426843159A43A5
:107360004260002901D0346006E08034A8686A6871
:10737000C0018018A042E4D8002038740846F8BD47
:10738000542D002050C300000020024005484168F1
:1073900002221143416041680122114341600020F3
:1073A0007047000000200240F8B50E4617460B4C0F
:1073B000207C012808D0012020740948FFF71CFA1E
:1073C0000025002802D006E00220F8BD6561376084
:1073D0000348FFF711FA2574F8BD0000542D002072
:1073E00050C3000012494868C0070DD0EFF3108069
:1073F00072B6104ACA60104ACA6080F310884868A2
:10740000C00701D001207047486880070DD5EFF311
:10741000108072B6094A0A61094A0A6180F310882D
:107420004868800701D501207047002070470000A0
:1074300000200240EFCDAB8905040302BFAE9D8C56
:1074400016151413F0B50022002961D001239340D2
:107450009E460B40002B57D095082E4CAD002D19A1
:10746000AC689607360F0F27B7403C40A44605246A
:107470002407A04201D1002419E0274CA04201D1E9
:10748000012414E0254CA04201D102240FE0244C39
:10749000A04201D103240AE0224CA04201D10424DD
:1074A00005E0214CA04201D1052400E00624B440AF
:1074B00064450FD11D4C26689E43266066689E4336
:1074C0006660E6689E43E660A6689E43A660AB6879
:1074D000BB43AB60046855000323AB401C4304600E
:1074E000D408A4002418266A5507EF0E0F25BD40C6
:1074F000AE432662C4689C43C46044687546AC438E
:10750000446084689C438460521C0B46D3409DD1E8
:10751000F0BD0000000001400004005000080050D1
:10752000000C005000100050001C005000040140EE
:10753000202805D103490020086003490120C871B3
:1075400070470000300000203C00002010B50449C6
:107550004A69024202D04861FFF7EAFF10BD00000D
:1075600000040140F0B400220B68002B6FD001270B
:107570000B6897403B40002B6AD00C79A407A40FFE
:10758000012C01D0022C10D1856854000326A6409E
:10759000B543CE68A6402E4386604468BC430D794F
:1075A000ED06ED0F9540254345600C79E443A407B3
:1075B00008D0C56854000326A640B5438E68A6408F
:1075C0002E43C6600C79A407A40F022C0CD1D4085A
:1075D000A40027183D6A5407E40E0F26A640B543C1
:1075E0000E69A6402E433E62056854000326A6405D
:1075F000B5430E79B607B60FA6402E4306604C6819
:10760000A403A40F50D02C4C656B01263543656351
:1076100095082A4CAD002F19BD689407240F0F263A
:10762000A640B54305263607B04201D100261BE02F
:10763000234EB04201D1012616E0224EB04201D1C4
:10764000022611E0204EB04203D103260CE030E0C8
:107650002AE01E4EB04201D1042605E01C4EB04285
:1076600001D1052600E00626A6402E43BE60194D36
:10767000AC689C434E68F60200D51C43AC60EC68D5
:107680009C434E68B60200D51C43EC606C689C437A
:107690004E68B60300D51C436C602C689C434E6852
:1076A000F60300D51C432C60521C0B68D34000D05D
:1076B0005DE7F0BC70470000001002400000014090
:1076C0000004005000080050000C00500010005052
:1076D000001C0050000401400069084201D0012054
:1076E000704700207047002A01D081617047816295
:1076F0007047000001488068704700007002002059
:1077000004494A6B01231A434A6303494A68024306
:107710004A60704700100240000001400248816842
:1077200002788918816070477002002010B500242B
:1077300007480168402211430160032000F00AF865
:10774000002801D0012401E000F080F9204610BD9E
:107750000020024070B504460E4D7D202978C000FF
:10776000FDF7C6FC01460C480068FDF7C1FC00F0BF
:1077700061FF002801D0012070BD042C07D2002237
:107780002146501E00F08AF96C60002070BD012077
:1077900070BD0000700200207C020020704770471E
:1077A0000E480F4AC16A491CC162016B491C016342
:1077B000538F00228B4202D20121416300E04263D9
:1077C000084B1878012807D107480168491C016057
:1077D000022901D302601A707047000000000020E7
:1077E000EC07002040000020640000207047704734
:1077F00070472030807B704710B5044620680168D0
:10780000C943C90708D18168C943C90704D1012107
:1078100041602046FFF7C4FF20680168C94389071B
:1078200008D48168C943890704D4022141602046F5
:10783000FFF7B4FF20680168C943490708D481688D
:10784000C943490704D404214160204600F0FCF8F4
:1078500020680168C943090708D48168C94309073A
:1078600004D4082141602046FFF7C0FF206801686A
:10787000C943C90608D48168C943C90604D4102184
:1078800041602046FFF78BFF20680168C9438906E5
:1078900008D48168C943890604D420214160204668
:1078A000FFF7A6FF20680168C943490608D481682C
:1078B000C943490604D4402141602046FFF797FFA1
:1078C00010BD0000F8B50446002C06D060682546BF
:1078D0002035A87B002802D006E00120F8BD00205A
:1078E0006873204600F046F80220A873206884469A
:1078F000C0686168012904D00122A36AD2059342BD
:1079000001D11E229043184B62699A4201D0174B55
:107910001840174B1840A368676A266A0B433E431A
:107920001E43A36A1E433043002903D12769E66939
:107930003E433043012903D00121C9058B4203D1C5
:107940002369E1681943084307498A4205D0A169C0
:107950000A43E1690143104608436146C8600120BB
:10796000A8730020F8BD0000FFFF00003F1FFFFFCD
:10797000FEF119FF10B50068084988420CD108488B
:10798000816BC20411438163002211460D2000F077
:1079900085F80D2000F076F810BD0000007C004056
:1079A000001002400068C06970470000F8B5044646
:1079B000164602222046203005468273214802687E
:1079C000C3041A4302602068C2689B121A43C26053
:1079D0002068026901273A43026122681020506042
:1079E000206881611021204602F07EFB032822D00E
:1079F000216808204860206846610821204602F07E
:107A000073FB032819D0204602F0F4FA2046FFF752
:107A1000F0FE032813D02068816839438160206814
:107A20000169394301612068016904221143016140
:107A3000AF730020F8BD0320F8BD0320F8BD03207C
:107A4000F8BD000000040140704700000448416B8D
:107A5000012211434163816B02041143816370472A
:107A600000100240002809DBC106C90E0120884031
:107A700003490860BFF34F8FBFF36F8F704700005B
:107A800080E100E0002805DBC106C90E0120884026
:107A9000014908607047000000E100E08207D30E52
:107AA000FF229A408907090E9940002808DB8308C5
:107AB00009489B001818036893430B430360704701
:107AC0000007000F0838830804489B001818C36992
:107AD00093430B43C361704700E400E000ED00E016
:107AE0000248016882151143016070470070004030
:107AF000F0B4164E326875152A40154B1B6ADB0729
:107B0000DB0F002A04D0002B02D03468AC43346071
:107B10003468A408A400044334600E4F3C69042078
:107B200004433C6101290ED040BF20BF20BF39690A
:107B300081433961002A04D0002B02D030682843E9
:107B40003060F0BC704730BFF1E7000000700040CB
:107B50000000014000ED00E0F8B504460026207862
:107B60005E4D80067DD55E48806BC00005D45C48C4
:107B7000816B02041143816301265A480168C905DB
:107B800017D40068FF210131084356490860FFF708
:107B9000B1FD074653480068C0050AD4FFF7AAFDA7
:107BA000C01B642801D90320F8BD4E480068C005F9
:107BB000F4D54B4F3868032109050840626811402D
:107BC000814208D09003800F032804D138688003D5
:107BD00001D50120F8BD28690321090408400028C7
:107BE00024D00A40824221D0207880061ED5286900
:107BF00088432A690121C9040A432A612A698A4300
:107C00002A612861C00511D5FFF774FD009028692D
:107C100080050BD4FFF76EFD0099411A324881426E
:107C200001D90320F8BD28698005F3D520788006A6
:107C300011D560688103890F032905D13A680905C8
:107C40008A43084002433A602869032261681204AB
:107C5000114008432861012E03D1B96B30078143DD
:107C6000B9632078C00705D0E868A1688008800063
:107C70000843E8602078800705D5E8680C21884330
:107C8000E1680843E8602078400706D5E8680321EA
:107C90008902884321690843E8602078000706D5F7
:107CA000E86803210903884361690843E860208884
:107CB000C00506D5E968032000048143A06901439B
:107CC000E9602078000606D5E86803218904884326
:107CD000E1690843E8600020F8BD00004010024060
:107CE000001002400070004088130000F8B5044600
:107CF0000D46002C1BD076480068C007C00FA84274
:107D00001CD2734F38684008400028433860FFF7A2
:107D1000F1FC06463868C007C00FA8420ED0FFF736
:107D2000E9FC811B6B48814203D90320F8BD012087
:107D3000F8BD3868C007C00FA842F0D12078664F60
:107D4000800705D5F868F0218843A1680843F860EA
:107D50002078C00772D06068022808D003280BD0B2
:107D600001280ED03968890510D40120F8BD396882
:107D700089030BD40120F8BD3968890106D401209C
:107D8000F8BD3968490701D40120F8BDF9688908B0
:107D900089000143F960FFF7ADFC064660680228E0
:107DA0000FD0032820D0012831D0F8680007800FB9
:107DB00044D0FFF79FFC811B464881423AD90320FB
:107DC000F8BDF8680007800F022837D0FFF792FC53
:107DD000811B4048814201D90320F8BDF8680007A3
:107DE000800F0228F2D129E0F8680007800F0328ED
:107DF00024D0FFF77FFC811B3648814201D9032044
:107E0000F8BDF8680007800F0328F2D116E0F86883
:107E10000007800F012811D0FFF76CFC811B2D4853
:107E2000814201D90320F8BDF8680007800F0128BE
:107E3000F2D103E0F8680007800FBAD12448016846
:107E4000C907C90FA9421CD9006821494008400050
:107E500028430860FFF74EFC06461D480068C0072F
:107E6000C00FA8420DD0FFF745FC811B1948814285
:107E700001D90320F8BD16480068C007C00FA8420A
:107E8000F1D12078400706D5F86807210902884318
:107E9000E1680843F8602078000707D5F8680721F3
:107EA000C90288432169C9000843F86000F042F81C
:107EB000F9680A4A0906090F515CC8400849086078
:107EC00008480068FFF746FC0028D3D1F8BD000041
:107ED0000020024088130000001002407EEB0008E2
:107EE0007C020020740200200148006870470000F6
:107EF0007C02002000B5FFF7F7FF0449C968044A77
:107F00004905490F515CC84000BD00000010024007
:107F100097EB000800B5FFF7E7FF0449C968044A7A
:107F20008904490F515CC84000BD000000100240A8
:107F300097EB000870B5214EF2680C2110460840FE
:107F40001F498B0004280CD04D00082810D00C28A5
:107F500010D070680004410F491C0120C003884004
:107F600070BD3068C00601D5084670BD184670BDAA
:107F7000284670BD9002134C000F205C1202940F33
:107F8000641CF268D20307D5294605F070F8224632
:107F90000023FDF7C3F870BD3268D20606D505F0A0
:107FA00066F822460023FDF7B9F870BD194605F0C2
:107FB0005EF822460023FDF7B1F870BD00100240C4
:107FC00000093D008EEB0008F0B583B00446002C9C
:107FD0000FD0F84EF5680C200540F768012000042A
:107FE00007402078C0075BD0082D09D00C2D03D0A6
:107FF0000FE0012003B0F0BD01200004874208D14A
:10800000306880034CD56068002849D1012003B056
:10801000F0BD012061680004814203D13168014351
:10802000316015E0052301221B049204994206D118
:1080300031681143316031680143316008E03168D3
:108040008143316031680140019130689043306074
:108050006068002812D0FFF74DFB02903068800363
:108060001ED4FFF747FB0299401A642802D9032067
:1080700003B0F0BD30688003F3D511E0FFF73AFBA1
:108080000290306880030BD5FFF734FB0299401A49
:10809000642802D9032003B0F0BD30688003F3D414
:1080A0002078800768D5E068810604D532682021F1
:1080B0000A43326088430923042D17D00C2D01D1C7
:1080C000002F13D0002842D031689943014331601A
:1080D000FFF710FB0746306840072FD4FFF70AFB75
:1080E000C01B022827D9032003B0F0BD316849071F
:1080F00001D500281CD071681F2212029143226909
:108100001202114371603168994301433160FFF7F6
:1081100011FFF16809060A0FA749895CC840A74901
:108120000860A7480068FFF715FB0028DCD123E0B2
:10813000012003B0F0BD30684007CFD570681F2123
:1081400009028843216909020843706014E030681D
:10815000400840003060FFF7CDFA0746306840071E
:108160000AD5FFF7C7FAC01B022802D9032003B0C3
:10817000F0BD30684007F4D42078C0066BD5002DE0
:1081800015D0A069002850D03068FF210131084384
:108190003060FFF7AFFA07463068800536D4FFF746
:1081A000A9FAC01B02282ED9032003B0F0BD306805
:1081B000800502D5A069002822D0706807214903F4
:1081C0008843216A084370607068217F0002000ABA
:1081D000090608437060206A410B491C0120C00356
:1081E0008840F16809060A0F7349895CC8407349E1
:1081F000086073480068FFF7ADFA0028D5D12AE07F
:10820000012003B0F0BD30688005C8D57068072133
:1082100049038843216A084370607068217F000227
:10822000000A09060843706015E03168FF2001303C
:1082300081433160FFF75EFA0746306880050AD552
:10824000FFF758FAC01B022802D9032003B0F0BD83
:1082500030688005F4D420785A4F00072FD5606924
:10826000002816D03869012108433861FFF742FA27
:1082700002903869800722D4FFF73CFA0299401A2D
:10828000022802D9032003B0F0BD38698007F3D576
:1082900015E03869400840003861FFF72BFA02907A
:1082A000386980070BD5FFF725FA0299401A022892
:1082B00002D9032003B0F0BD38698007F3D42078D9
:1082C000400775D500200190B06BC00006D4B06B9C
:1082D000012109070843B063012001903A48016871
:1082E000C90519D40068FF210131084336490860E7
:1082F000FFF700FA029034480068C0050CD4FFF77D
:10830000F9F90299401A642802D9032003B0F0BD9C
:108310002D480068C005F2D5FF20A26801308242D6
:1083200003D13969014339611BE001218902002A27
:108330000AD005231B029A420DD13A690A433A61D9
:108340003969014339610CE03A6982433A6138691D
:108350008843386105E03A6982433A613869884365
:108360003861A068002813D0FFF7C4F9029038697B
:10837000800530D4FFF7BEF90299411A13488142B3
:1083800002D9032003B0F0BD38698005F2D522E0A0
:10839000FFF7B0F90290386980051CD5FFF7AAF9FC
:1083A0000299411A0948814212D9032003B0F0BD55
:1083B00019E00000001002407EEB00087C02002063
:1083C000740200204010024000700040881300003A
:1083D00038698005E2D40198012804D1B06B0121ED
:1083E00009078843B063606A002864D00C2D49D027
:1083F00001252D0602280FD03068A8433060FFF712
:1084000079F904463068800155D5FFF773F9001BF0
:10841000022833D90320C9E73068A8433060FFF74A
:1084200069F907463068800109D5FFF763F9C01B79
:10843000022801D90320B9E730688001F5D4E16A48
:10844000A06AF2680843216BFD231B049A43114381
:108450000843F060306828433060FFF74BF904466A
:108460003068800127D4FFF745F9001B022801D9A5
:1084700003209BE730688001F5D51CE0306880015F
:10848000C3D418E0012814D0F06801210904A26ABD
:10849000014091420BD10F218904E26A01409142CF
:1084A00005D1032189050840216B884203D00120B2
:1084B0007CE701207AE7002078E7000002480169A4
:1084C000022211430161704700E000E070B50446EC
:1084D000002C10D0022025464035687420680168C1
:1084E000402291430160204600F064F8002060655E
:1084F0006874287470BD012070BDF8B50446002C66
:108500000ED0FF27606A0537002600280AD02661B2
:108510006661A66225464035687C002807D00AE0DF
:108520000120F8BD6068B842F3D0E661F1E72E742F
:10853000204600F053F80221697420680268402345
:108540009A4302602123A26860689B021A40384067
:108550001043E3688A021340184323690B40217DCE
:108560001843C907C90F0843A1699310194008436C
:10857000E169382319400843216A802319400843E0
:10858000A16A93001940084321680860A06904218A
:10859000000C0840616A10231940084321684860B4
:1085A0002068C1699143C16166650120687400203B
:1085B000F8BD000010B500680649884209D1064898
:1085C000416B8214914341630520E0210007FEF7CF
:1085D00039FF10BD003001400010024010B586B0D8
:1085E000044614216846FCF7E2FD104920688842E1
:1085F00019D10F48416B821411434163C16A0122B2
:108600001143C162C06A002110400590E020009033
:1086100002200190032003900291049105206946F5
:108620000007FEF79FFF06B010BD000000300140BC
:108630000010024010B40B49401E884202D910BC01
:10864000012070470849486108480723C26912029F
:10865000120A4C042243C261002088610B6110BCE5
:1086600070470000FFFFFF0000E000E004ED00E0C5
:1086700002480169022291430161704700E000E075
:10868000F0B402462032137E012B22D0012616764A
:108690000223537603685D689C687027BD430F68AA
:1086A0002F435F600068B307984208D00A4B984296
:1086B00005D00A4B984202D0094B984204D180233E
:1086C0009C43496821438160567600201076F0BCB7
:1086D0007047F0BC022070470004004000080140D1
:1086E0000014014010B5022104462034617601686F
:1086F0000A6A094B1A4203D10A68520852000A60FA
:1087000000F02CF80020A077A076E0762077607744
:108710006076207610BD00001111000070B505468E
:10872000002D05D02C462034607E002802D006E0C3
:10873000012070BD00202076284600F01DF80220A0
:108740006076291D286803F019FB0120A077A07628
:10875000E076207760776076002070BD006804497D
:10876000884204D10348416B04229143416370471E
:10877000000801400010024000680449884204D10A
:108780000348416B042211434163704700080140D4
:1087900000100240014620314A7E012A01D001200A
:1087A000704702224A760168CB6801221343CB60EE
:1087B00000689107884208D00B49884205D00B49D0
:1087C000884202D00A49884208D181684907490F86
:1087D000062906D001681143016002E001681143D7
:1087E00001600020704700000004004000080140C4
:1087F000001401400168CA6852085200CA6001684A
:108800000A6A064B1A4203D10A68520852000A60EB
:108810000121203041760020704700001111000036
:10882000F8B50446002625462035287E012817D0B5
:108830000120287602206876206882687727BA436C
:10884000FF231B029A4382600868502838D00EDC50
:10885000202853D006DC002850D010281ED14DE02F
:108860000220F8BD302849D0402817D13CE06028CC
:1088700030D0702819D001221203801A0FD09042F4
:108880000CD1CB684A688968206803F0B9FA20687F
:108890008168012292031143816000E001260120DA
:1088A0006876002028763046F8BDCB684A6889682B
:1088B000206803F0A5FA2068816839438160EEE7FB
:1088C000CA684968206803F020FB5021206803F043
:1088D000A3FAE4E7CA684968206803F028FB60212E
:1088E000206803F099FADAE7CA684968206803F05B
:1088F0000CFB4021206803F08FFAD0E72268014684
:10890000104603F089FACAE710B586B00446142170
:108910006846FCF74CFC0D492068884213D10C488E
:10892000C26A02210A43C262C06A019108400590EE
:1089300008030090002002900390062004906946EE
:108940000448FEF70FFE06B010BD0000000801400D
:108950000010024000040050F8B504460D46002700
:1089600026462036307E01280ED001203076002A9F
:108970000CD0042A1ED0082A33D00C2A45D0012757
:10898000002030763846F8BD0220F8BD2946206820
:1089900003F04AFA20688169082211438161206846
:1089A000816904229143816120688169EA681143E9
:1089B0008161E5E72946206803F04FFA2068826963
:1089C0000121C9020A438261206881690122920261
:1089D0009143816120688169EA68120211438161D3
:1089E000CEE72946206803F055FA2068C1690822BD
:1089F0001143C1612068C16904229143C1612068AB
:108A0000C169EA681143C161BAE72946206803F0E9
:108A10005DFA2068C1690122D2021143C161206858
:108A2000C269012189028A43C2612068C169EA687A
:108A300012021143C161A3E770B50546002D05D0B0
:108A40002C462034607E002802D006E0012070BD54
:108A500000202076284600F00FF802206076291DBD
:108A6000286803F08BF90120A077A076E0762077C4
:108A700060776076002070BD7047000070B50546D5
:108A80002C462034002908D0042908D0082908D011
:108A9000627F012A07D0012070BDA27EF9E7E27E45
:108AA000F7E7227FF5E70220002920D0042920D013
:108AB000082920D060770122286803F093F901216A
:108AC000286889070122884208D00E49884205D0CB
:108AD0000D49884202D00D4988420ED1816849076C
:108AE000490F06290CD001681143016008E0A07607
:108AF000E1E7E076DFE72077DDE701681143016019
:108B0000002070BD00040040000801400014014036
:108B100070B504460D4600222946206803F062F92C
:108B20002068016A0B4A114203D1016849084900D3
:108B3000016001202034002D06D0042D06D0082D20
:108B400006D06077002070BDA076FBE7E076F9E7FD
:108B50002077F7E7111100007047704770B50446A1
:108B6000002C1BD02420E0672068016849084900D8
:108B700001602068002505602068456020688560E8
:108B8000204600F09BF9204680304560E56705608F
:108B90002566656660342576002070BD012070BDB5
:108BA00010B504F093F810BDF8B504462268D069FA
:108BB00011689368A24D06462E40002E09D1850605
:108BC00007D58D0605D5A16E002901D0204688471E
:108BD000F8BD25468035002E7FD09A4FDE07F60F70
:108BE0000F40374379D0C70706D0CF0504D50127FA
:108BF00017626A683A436A60820708D5DA0706D0C6
:108C0000276802223A626A6804273A436A60420788
:108C100008D5DA0706D0236804221A626A6802239C
:108C20001A436A60020709D520220A40324305D060
:108C3000236808221A626B6813436B60020509D52A
:108C40004A0107D501222368D2021A626A682023EA
:108C50001A436A606A68002ABAD0800606D5880678
:108C600004D5A16E002901D0204688476868216894
:108C70008968490602D42821084228D0204603F0FA
:108C80001DFB2068816849061DD5EFF31081012284
:108C900082F31088836840229343836081F31088B5
:108CA000606F00280BD068498163606FFEF7BDFAE2
:108CB00000288DD0606F816B8847F8BD0DE020469D
:108CC000FFF76EFFF8BD2046FFF76AFFF8BD2046AC
:108CD000FFF766FF00206860F8BD266E012E7DD18B
:108CE000C6067BD5CE0679D510231362206881682D
:108CF00026464906403600294CDA626F11684968F9
:108D000089B20029E8D0378B8F42E5D97183116889
:108D10000968890634D4EFF31081012282F31088A8
:108D200002681F01BA43026081F31088EFF31081DB
:108D3000012080F310882068826852085200826007
:108D400081F31088EFF31081012080F310882068F0
:108D500082684027BA43826081F31088202028600F
:108D600000202066EFF31081012080F31088206836
:108D700002689A43026081F31088606FFEF731FA4F
:108D800002206066308B718B401A81B22046FFF75B
:108D9000E3FEF8BD318B728B891A89B2728B002A7F
:108DA000F7D00029F5D0EFF31082012686F3108862
:108DB0000668FF272137BE43066082F31088EFF371
:108DC0001082012080F3108820688668760876007B
:108DD000866082F310882020286000E013E00020E5
:108DE0002066A066EFF31082012080F310882068CF
:108DF00005689D43056082F3108802206066204666
:108E0000FFF7AAFEF8BDC50208D55B0206D5012012
:108E1000000510622046FFF7A0FEF8BD020607D548
:108E20000A0605D5E16E0029F7D020468847F8BD2F
:108E30004006FCD54806FAD5204603F06FFAF8BD87
:108E40000F080000200100044DC1000810B50446C1
:108E5000002C03D0E06F002802D007E0012010BDF5
:108E6000002178200155204600F064F82420E067B6
:108E700020680168490849000160204603F050FB62
:108E8000012819D0606A002802D0204603F090F82B
:108E9000206841680922D2029143416020688168BC
:108EA0002A229143816020680168012211430160F8
:108EB000204603F0E3F810BD012010BD10B5026894
:108EC0001748184982420BD1886B012292049043C3
:108ED0008863032189021448FEF7B4FA1D200EE0CE
:108EE000124B052000079A420CD14A6B01239B03C9
:108EF0009A434A6303214902FEF7A4FA1B20FEF7B6
:108F0000B1FD10BD0A4B9A42FBD18A6B01235B0471
:108F10009A438A630C21FEF795FA1C20EFE70000C4
:108F2000004800400010024000040050003801409A
:108F300000440040F0B587B0044614216846FCF7B1
:108F400036F9314A266800253048022103230424DB
:108F5000964218D1826B4E0432438263C26A0A433E
:108F6000C262C06A6A4608400590980223C218C2CD
:108F700069462748FEF7F6FA002211461D20FEF743
:108F80008DFD1D201CE0234F0122BE421CD1456BEC
:108F9000960335434563C56A1543C562C06A6D468D
:108FA00010400590032040021FC5052069460007B8
:108FB000FEF7D8FA002211461B20FEF76FFD1B209A
:108FC000FEF760FD07B0F0BD134FBE42FAD1866BCD
:108FD00001277F043E438663C66A1643C662C06AA1
:108FE0006E46C007C00F05900C2023C6052018C68A
:108FF00069460007FEF7B6FA002211461C20FEF76C
:109000004DFD1C20DCE7000000480040001002403D
:1090100000040050003801400044004070B5802337
:109020001B58202B01D0022070BD00290AD0002A35
:1090300008D0012483682403A34209D10369002BCB
:1090400002D005E0012070BDCB0701D0012070BD2A
:10905000002303660A4C0368A3420ED05C68240216
:109060000BD5EFF31084012585F310881D680126C8
:10907000B60635431D6084F3108803F08BFB70BD8A
:109080000048004070B580231B58202B01D00220DF
:1090900070BD00290AD0002A08D001248368240367
:1090A000A34209D10369002B02D005E0012070BD65
:1090B000CB0701D0012070BD002303660A4C036872
:1090C000A3420ED05C6824020BD5EFF31084012577
:1090D00085F310881D680126B60635431D6084F3AC
:1090E000108803F0AFFB70BD0048004010B503F0DE
:1090F0000FFE10BD7047FFB583B004460F461546FE
:10910000E06F202802D0022007B0F0BD002F0AD067
:10911000002D08D00120A168000381420BD12069F5
:10912000002803D007E0012007B0F0BDF80702D007
:10913000012007B0F0BD0021842001512120E0670B
:10914000FEF7D8FA02902646403635827582012015
:10915000A1680003814202D12069002813D03D4656
:109160000027708A00281CD00698009000228021D9
:109170002046029B03F036FC002806D02020E06742
:10918000032007B0F0BD0025EBE7002D18D02168C3
:10919000287888626D1C708A401E7082708A002850
:1091A000E2D106980090002240212046029B03F065
:1091B00019FC00280BD02020E067032007B0F0BD89
:1091C00038882168C005C00D8862BF1CE3E72020F5
:1091D000E067002007B0F0BD70B50446E06F2028BE
:1091E00001D0022070BD00290AD0002A08D0012336
:1091F000A0681B03984209D12069002802D005E02D
:10920000012070BDC80701D0012070BDE164204677
:1092100040300282428200214030054641602120D8
:10922000E067206F00281AD0154BC362236F1548E2
:109230001863236F14485863206F816320681346B6
:109240002830266F02463046E16CFEF714F80028FD
:1092500005D0102068602020E067012070BD2168E3
:1092600040200862EFF31081012080F3108820680D
:10927000826880231A43826081F31088002070BDC9
:1092800067C20008B3C2000861C1000830B4C36FF0
:10929000202B02D030BC0220704700290AD0002ABF
:1092A00008D0012483682403A3420BD10569002D53
:1092B00003D007E030BC01207047CD0702D030BC9E
:1092C00001207047C164014640310A824A82002170
:1092D000C166842211502121C167A34202D10169D4
:1092E000002910D00949C166EFF31081012282F3F1
:1092F00010880068026880231A43026081F3108896
:1093000030BC002070470249C166EDE787C90008FC
:1093100025C9000810B503F093FD10BD704700008B
:1093200000200149087070472805002001200149EC
:10933000087070472805002070B504460D46204689
:1093400000F02CF8012801D1801E70BD2268501C4D
:10935000E168FBF7CDFE2160236921685943A368CA
:10936000C81829462269FBF709FF0020EDE710B570
:109370008160C2600361012444600024046010BD68
:1093800010B504462268501CE168FBF7B1FE606826
:10939000814201D1012010BD0020FCE710B5044638
:1093A0002268901CE168FBF7A3FE6068814201D14E
:1093B000012010BD0020FCE770B504460D46204694
:1093C000FFF7DEFF012801D1801E70BD23696068B0
:1093D0005843A368C11828462269FBF7CFFE62688C
:1093E000501CE168FBF784FE61600020EDE770B57A
:1093F00004460D46002C01D1401E70BD00BF206800
:10940000A842FCD32068401B206062685019E168C4
:10941000FBF76EFE61600020EFE770B504460D4675
:10942000002C01D1401E70BD20684019206000BF93
:10943000E16820688842FBD8A2685019E168FBF710
:1094400057FEA1600020EEE7FFB581B004460D464F
:1094500016460027002E06D00498002803D0E168A5
:109460002068884203D30020C04305B0F0BD2168C6
:10947000E068401AA84202D20020C043F5E7A06885
:109480004019E16888420BD9A168E068471A216851
:10949000E068401AE919884202D20020C043E4E79C
:1094A000A268D019E168FBF723FE316079190498AE
:1094B00001600020D9E70146486870470146886886
:1094C00070470246002A01D1401E704700205060BC
:1094D00090601060D16000BFF7E70146002901D11C
:1094E000012070470868002801D10120F9E7002019
:1094F000F7E70146002901D1012070470A68C868D2
:10950000904201D10120F8E70020F6E70FB400B542
:109510000D48FFB0007882B0012805D000207FB050
:1095200002B008BC04B01847012183AB4902684669
:10953000829A03F06FFD6846FBF758FE02466946C3
:10954000002003F011FCEAE75C01002010B5064A98
:109550001278012A01D0002010BD0A4601460020E1
:1095600003F002FC10BD00005C0100200349096803
:109570000160022181710149086070479802002052
:1095800000BFEFF30580002800D07047074800684F
:10959000002804D1012080F3108800BF00BF0348D9
:1095A0000068401C0149086000BFEEE7800200200F
:1095B00070B504460D4600F04FF800280FD000F0BB
:1095C0004BF80B21C90140180069002807D000F0B2
:1095D00043F80B22D2018018016902A088470020BD
:1095E00070BD00001B5B481B5B4A000070B5024663
:1095F0000C4600210023002A01D0002C02D10020BB
:10960000C04370BD0021002316E0C8000D4D28584E
:10961000002810D1D8001058CD000A4E7051D80043
:1096200080184068CD00AD19686007480068401C8C
:10963000054D28605B1C491C502901D2A342E4D38C
:109640000020DEE7A4020020A002002001480068FC
:1096500070470000A0020020014800687047000029
:109660009C020020F8B506460F46002536E000248F
:1096700018E0FFF7F1FF002813D0FFF7EDFF0B21F3
:10968000C9014018006900280BD0FFF7E5FF0B2344
:10969000DB01C01802692819C000134B195813A028
:1096A0009047641C052C04DAFFF7D0FF2919884283
:1096B000DFD8FFF7D1FF00280FD0FFF7CDFF0B2138
:1096C000C90140180069002807D0FFF7C5FF0B2229
:1096D000D2018018016907A088476D1DFFF7B6FF0A
:1096E000A842C4D80020F8BDA4020020252D3136A0
:1096F000730000000D0A00000146202902D300205B
:10970000C0437047012218204843044B1A500022DE
:1097100018204843C01882600020F2E76C2D00201A
:1097200070B505460024002D01D1401E70BD0024F7
:109730000CE0182060430C490858002805D101218D
:1097400018206043084A115002E0641C202CF0D31A
:1097500000BF202C05D105A0FFF7D8FE0020C04394
:10976000E4E72C600020E1E76C2D002074696D6552
:10977000722049442069732066756C6C0D0A0000E4
:1097800010B5002400BF41E018206043214908586B
:1097900002283AD118206043401880681E490968A1
:1097A000091A182060431B4A8018C06881422CD9CE
:1097B00018206043114640184069002820D0182026
:1097C000604340180079002804D10121182060432B
:1097D00011500AE00221182060430E4A11500E4831
:1097E0000168182060438018816018226243094B89
:1097F000D218106918226243D2185169884704E0D0
:10980000012118206043034A1150641C202CBBD353
:1098100010BD00006C2D002088020020F0B5044629
:10982000059D202C02D30020C043F0BD0226182045
:1098300060430E4F3E50182060433E468019017130
:109840000B48066818206043C019866018206043E2
:109850003E468019C2601820604380194361182079
:109860006043801905610020DFE700006C2D0020B7
:109870008802002007480068401C06490860064826
:10988000026840680021521C484103490A60486050
:1098900070470000880200209002002000BFEFF314
:1098A0000580002800D0704709480068002804D0CF
:1098B00007480068401E06490860054800680028FF
:1098C00004D100BF80F3108800BF00BF00BFEAE7EB
:1098D0008002002070B504460D4629462046FBF75D
:1098E00066FC70BD0146302904DB392902DC0846DC
:1098F00030380EE0412904DB462902DC08463738BF
:1099000007E0612904DB662902DC0846573800E0DD
:109910000020C0B2704710B502460B46002406E096
:109920001078FFF7DFFF21014418521C5B1E002B4B
:10993000F6D1204610BD0FB4F0B585B00446002026
:10994000049000222020039000200290002C02D0DE
:109950000C98002805D1002005B0F0BC08BC04B06C
:1099600018470DA80490CFE0002908D10C98007882
:10997000252803D10C984078652800D0C9E00C98C0
:10998000007825286ED10C98401C0C900C9800781B
:1099900003900C98401C0C900398652877D004DC49
:1099A0002A2807D0642873D113E0702872D0782851
:1099B000F9D13EE008E020780C9B1B78984202D059
:1099C000641C491E00E001E00029F4D100BF521CD4
:1099D00088E0002601960096002300252020049EA2
:1099E00020CE049618E02078009E002E05D12D2868
:1099F00003D10126019600960CE0302809DB3928B6
:109A000007DC012600960A265E430746303FF3191D
:109A100000E003E0641C491E0029E4D100BF019E60
:109A2000012E01D1DE43731C002D00D02B60521C8F
:109A300058E000230025049E20CE04961FE02078E5
:109A4000302806DB392804DC1E010746303FF319B5
:109A500013E0612807DB662805DC1F010646573E38
:109A6000BB190AE043E0412806DB462804DC1F015D
:109A70000646373EBB1900E003E0641C491E00297E
:109A8000DDD100BF002D00D02B60521C2AE01BE06E
:109A900024E0FFE7049E01CE04960025002325461E
:109AA00009E026780C9F3F78BE4201D05B1C00E0A5
:109AB00003E0641C491E0029F3D100BF002801D037
:109AC00005604360521C0DE0049B01CB0493002809
:109AD00000D00460521C0123029303E00120029095
:109AE000002200BF00BF029801280DD111E02078AC
:109AF0000C9B1B78984205D1641C0C98401C0C9060
:109B0000491E01E0002204E00C980078002800D0F3
:109B10002AE700BF0020049010461DE70FB4F8B5F7
:109B200006460C46002509A8009021463046009BB9
:109B3000089A03F06FFA054600200090A54200D372
:109B4000651E2846F8BC08BC04B01847FEB504469C
:109B50000F4615460026002001900090002C01D0F1
:109B6000002D01D10020FEBD2846FBF73FFB0090F1
:109B70000098874201D20020F5E70098381A01903A
:109B8000002609E0A0192946009AFBF736FB0028B9
:109B900001D1A019E7E7761C01988642F2D3002094
:109BA000E1E770B504460D46002C01D0002D02D12E
:109BB0000020C04370BD012120461030FFF717FC84
:109BC00020462030A968FFF712FC0020F2E770B5AC
:109BD00004460D46002C01D0002D02D10020C043C8
:109BE00070BD012120461030FFF717FC20462030C1
:109BF000A968FFF712FC0020F2E710B50446002C1C
:109C000000D110BD20461030FFF767FC012801D1BC
:109C10000020F6E720462030FFF75FFC012801D145
:109C20000020EEE720461030FFF745FC0C214843AA
:109C300021684018E5E77CB504460E460025002063
:109C400001900090002C00D17CBD20461030FFF721
:109C500050FC002801D00020F6E76B4601AA3146EF
:109C600020462030FFF7F0FB002801D00020EBE772
:109C700020461030FFF722FC0C214843216845188C
:109C8000A0680199401828606E600098A860284676
:109C9000DAE7FFB581B004460E461D4600270C20CA
:109CA00068430399884202D3781E05B0F0BD0C20AA
:109CB0002F4647432660676060688019A06003985C
:109CC000C11BE160294620461030FFF7FAFB204611
:109CD0002030E168FFF7F5FB0020E6E7FEE7000033
:109CE00010B50E4C002208212046FDF7FCFC002296
:109CF00010212046FDF7F7FC0A2003F0C6FF0122E1
:109D000008212046FDF7EFFC0A2003F0BEFF0022E9
:109D100008212046FDF7E7FC10BD000000040050BC
:109D200010B50E4C002208212046FDF7DCFC012274
:109D300010212046FDF7D7FC0A2003F0A6FF0122E0
:109D400008212046FDF7CFFC0A2003F09EFF0022E9
:109D500008212046FDF7C7FC10BD0000000400509C
:109D6000F8B50024144E0746254600220821304647
:109D7000FDF7B9FC0A2003F088FF012208213046D4
:109D8000FDF7B1FC6006040E10213046FDF7A4FC7F
:109D9000002801D0641CE4B2052003F076FF6D1C9E
:109DA000EDB2082DE1D3002F03D0FFF799FF204635
:109DB000F8BDFFF7B5FFFAE70004005070B5154E87
:109DC0000546002208213046FDF78DFC0024E809F5
:109DD00001D0012200E0002210213046FDF783FC73
:109DE0006806050E0A2003F050FF012208213046C4
:109DF000FDF779FC0A2003F048FF002208213046D5
:109E0000FDF771FC0A2003F040FF641CE4B2082C4B
:109E1000DDD370BD0004005010B50C4C01221021A0
:109E20002046FDF760FC012208212046FDF75BFC7F
:109E3000002210212046FDF756FC0A2003F025FFE2
:109E4000002208212046FDF74EFC10BD0004005002
:109E500010B50E4C002208212046FDF744FC0022DC
:109E600010212046FDF73FFC0A2003F00EFF0122DF
:109E700008212046FDF737FC012210212046FDF77E
:109E800032FC0A2003F001FF10BD00000004005066
:109E900070B5144D0024012210212846FDF723FC43
:109EA000062003F0F2FE012208212846FDF71BFCE4
:109EB000062003F0EAFE07E0641CE4B2FA2C03D9A2
:109EC000FFF7C6FF012070BD10212846FDF704FCF6
:109ED0000028F1D1002208212846FDF704FC0020CB
:109EE00070BD00000004005010B5FCF723FA10BD4F
:109EF00010B53721202000F070F80321212000F058
:109F00006CF84021222000F068F80821232000F09E
:109F100064F8AA21302000F060F80A480221018785
:109F2000322000F05AF80121332000F056F85F216A
:109F3000202000F052F8044800F008F80A2003F04E
:109F4000A4FE10BDEC0700202B02002010B5014636
:109F50000F2000F021F8002800D0012010BD10B51E
:109F60000446FFF759FF3220FFF728FFFFF790FF65
:109F7000E0B2FFF723FFFFF78BFFFFF74DFF332022
:109F8000FFF71CFFFFF784FF0020FFF7E9FE044600
:109F9000FFF75EFF204610BD10B50C46FFF7DFFF50
:109FA0002070012010BD70B50D460446FFF734FF48
:109FB0003220FFF703FFFFF76BFFE0B2FFF7FEFE73
:109FC000FFF766FF2846FFF7F9FEFFF761FFFFF78F
:109FD0003FFF0A2003F059FE70BD10B5FFF7E3FF05
:109FE000012010BD10B50248FDF706FC10BD0000B1
:109FF0008C050020F0B583B004460026EFF31080F6
:10A000000090012080F31088344B2068C21804D1DE
:10A010003349CE68032189040E4081680291C168EA
:10A02000019141698569002A07D12E48826AC704D7
:10A030003A438262826ABA438262084628433CD02D
:10A0400026482268C24205D12548C36803229204EB
:10A050009343C36027462037002910D02068026947
:10A0600001231A430261206841610821204600F063
:10A070003BF8032800D1B873216808204860002D00
:10A0800010D02068016901221143016120688561B7
:10A090001021204600F028F8032800D1B873216869
:10A0A000102048600D482168C14206D10C48C168A3
:10A0B0000322920491433143C16020680169490839
:10A0C0004900016121680298886021680198C86090
:10A0D000009880F3108803B0F0BD00000084FFBF3B
:10A0E000401002400010024070B506460D460024A4
:10A0F0000B480A490068FAF7FBFF7D21C900484375
:10A100003268401E002800D1032413682946994371
:10A1100001D00028F5D1204670BD0000204E00007F
:10A120007C02002010B50248FEF73EFD10BD000085
:10A13000BC05002010B5032000F002F810BD00009F
:10A1400070B5164D00262C460C3C002811D0214637
:10A150004978032814D001280AD1491CC8B260707C
:10A160000C2817D204280FD08000285800F0BEF821
:10A1700070BD00F045F90520FDF7B6F8667001E006
:10A180000029F5D12868F1E705492869096800F038
:10A19000ADF870BD00F02AF970BD0000F401002098
:10A1A0006800002000B587B0012069464870022091
:10A1B00008700E490191410202910D4903918021DD
:10A1C000049105906946012002F0B6FC0948FFF7AA
:10A1D000A7FA00F015F900F079F86420FDF784F88B
:10A1E0000020FFF7ADFF002007B000BDBC26002017
:10A1F000BC2A0020EC010020032802D30020C04329
:10A200007047C3000248C150181882800020704770
:10A21000A426002008B500206946087003E06846BF
:10A22000007800F007F86946012002F045FC00289C
:10A23000F5D008BD70B51E491E4B0A78012A05D11C
:10A240008A687F2A02D29854521C8A6000220A2807
:10A2500002D00D2804D029E001208A60087025E092
:10A260000A708C68002C21D018192038C277114D43
:10A270004868FFF741FA10A221462846FFF766FC1E
:10A28000002805D029460DA0FFF740F901200BE07A
:10A290000CA221462846FFF759FC002806D0294683
:10A2A00006A0FFF733F90220FFF74AFF002070BD38
:10A2B000E80100203C2B00206F6B00005B525D200A
:10A2C00025730A006572726F7200000010B50348B2
:10A2D000012281880068FDF706FA10BDA42600203F
:10A2E00010B50020FFF72CFF10BD00000FB430B5F3
:10A2F00091B015AB402101A8149A02F08BFE002505
:10A3000001A8FAF773FF024601A9012002F02CFD13
:10A3100004460A487D220095074B1201002140683F
:10A32000FFF77CFA01A906A0FFF7F0F8204611B06C
:10A3300030BC08BC04B0184735A10008E801002073
:10A340005B535D2025730A0070B505460C480C462A
:10A3500040780C2802D00020C04370BD00F050F8B7
:10A360000520FCF7C1FF22462946012002F0FCFC33
:10A370000520FCF7B9FF00F039F8002070BD00009F
:10A38000E8010020F8B5124D124C28682169401AE6
:10A3900006281CD9012020710B210F48FFF7D4FF9C
:10A3A000286820610D4CFF2121600D4D0D4E0E4F90
:10A3B0002B683268386801F049F96420FCF794FF93
:10A3C000002121602B683268386801F03FF9F8BD40
:10A3D0002C0000203C000020680100202400002008
:10A3E0001C000020200000202800002010B5034899
:10A3F000002281898068FDF776F910BDA42600202F
:10A4000010B50348012281898068FDF76CF910BD01
:10A41000A42600201CB5002118480091164A01917D
:10A420000260C163120542608160072282630122DB
:10A4300002610246C16020321170FF235170C233A5
:10A44000436281621173016381610422416342614D
:10A45000C161FCF7EDFC002801D072B6FEE70848A8
:10A4600000908013019069460448FCF733FC0028F3
:10A4700001D072B6FEE71CBD00240140300500206B
:10A4800002000004F0B587B014216846FAF78FFE89
:10A490004148C26A04210A43C262C26A0A40059264
:10A4A000C16A01252943C162C16A29400591C26A76
:10A4B00002210A43C262C06A052708403F0705908F
:10A4C000002236493846FDF70EF900223449354856
:10A4D000FDF709F9012211033846FDF704F90122BD
:10A4E00040213048FDF7FFF8112636040024694664
:10A4F0003846019600950294FDF734F82A480090FA
:10A5000002946946019503943846FDF72BF82448D8
:10A510000294183800906946019503942148FDF78C
:10A5200021F8A22000906946019602941D48FDF78B
:10A5300019F8092000030090019469460294194813
:10A54000FDF710F818200090112001900294694640
:10A5500003941448FDF706F8402000900320039070
:10A560000195029469460F48FCF7FCFF2802FDF7AD
:10A57000C7F8002211460520FDF790FA0520FDF7E7
:10A5800081FA002211460720FDF788FA0720FDF71F
:10A5900079FA07B0F0BD00000010024010890000F9
:10A5A0001D410000000400501099000010B5FFF795
:10A5B00031FF00F009F800F099F800F0B3F800F06E
:10A5C0001FF800F043F810BD10B50C480A490160AF
:10A5D000E1214902416000218160C1600161816126
:10A5E0000C22016242614162FEF730FC002801D07A
:10A5F00072B6FEE710BD000000480040BC05002018
:10A6000010B5114C0F482060FF200530606000201D
:10A61000A060E06020616061E06101212062490288
:10A620006062A161A0620720E0622046FDF765FF3D
:10A63000002801D072B6FEE720680168402211436D
:10A64000016010BD003001405407002010B58AB0F1
:10A6500000240494059406940794089422480994CD
:10A660000094019402941F49039401601F218460A7
:10A6700041600461F9214461C160FEF74FF8002890
:10A6800001D072B6FEE701200003049004A9164829
:10A69000FEF7C6F8002801D072B6FEE71248FEF7B2
:10A6A000CBF9002801D072B6FEE7089408A90E483D
:10A6B0000994FDF7E5FF002801D072B6FEE760209F
:10A6C0000090019402940022694603940648FEF724
:10A6D00043F9002801D072B6FEE70348FEF714F9EB
:10A6E0000AB010BD00080140AC07002010B50C48AE
:10A6F0000A490160E1214902416000218160C16095
:10A7000001618161C1610C22016242614162FEF717
:10A710009DFB002801D072B6FEE710BD0038014055
:10A720004406002010B50C480A4901604B21C901BC
:10A73000416000218160C16001618161C1610C22C1
:10A74000016242614162FEF781FB002801D072B6CE
:10A75000FEE710BD00440040CC060020FEE70000EC
:10A76000F0B58BB00A2003F0B0FD7D20400103F06E
:10A77000C7FDFF4C00256570FE48E064607C0C2836
:10A7800001D30B20607420790A2801D90A20207196
:10A79000A570207D0127002803D0032801D027764B
:10A7A00000E02576F448F54E00783071F4480078E2
:10A7B000F071E06AF070010A3172401CE0622079A9
:10A7C000B07442003046EF491330FAF7D7FC2079D5
:10A7D000EC4982004000801960311330121DFAF7F5
:10A7E000CDFC2079062142004843E6498019EC312E
:10A7F0001730921CFAF7C2FCE3490020085E0028DB
:10A8000003D0E24A128A101808802079DB4EC30078
:10A8100098190A7842764978817616207072B57256
:10A82000A07F3073D2493046203113380A78027540
:10A830004978417518461D300022314603F030FE3C
:10A8400020790021C0001D3003F03CFE02F0C2FB65
:10A85000022003F08BFDF571A574A573012020740F
:10A86000E573CB48FDF79EF8A0840646A5702079D5
:10A87000FAF782FFC74AC84BFAF76CFE03F080F97B
:10A880000022C64BFAF7B4FDFAF7BCFF0006C00C75
:10A89000801980B20121C903E084884201D3401AA3
:10A8A000E084BF48A063E078401CE070B848FDF742
:10A8B00079F8B44E6084A43E304622300890001FE0
:10A8C0000290001F0190801E079036E1B048FDF70E
:10A8D00069F86084B34F0BE0AD48FDF763F880B2D0
:10A8E0006084E18C884203D3AF4A8918884206D33A
:10A8F00000210F2003F056FC38422063ECD0206B7F
:10A90000411C21D040047DD58122D20100210F209D
:10A9100003F09BFD0021102003F044FC4106994800
:10A92000490E27460022A438A16403F08BFC03F0F3
:10A930004DFC3865002003F0E3FC002003F09BFC95
:10A94000717A1729C1D101E002F0C6FB02229749B2
:10A95000701DFAF752FC0028B7D103F0ECFDF96541
:10A96000B86503F0D5FD79663866B8786946401C4D
:10A97000B8708448AB38027A0A70407A4870088808
:10A980000990398C88427ED17E490320903108702D
:10A9900008980090236E0020029A019900F07CFE36
:10A9A0007648834F8C30C08E388074488C30008F4E
:10A9B000A0837748FCF7F6FF608403F011FBF07C7E
:10A9C0000009607513D002227849701DFAF715FC52
:10A9D00000280CD101206949A074C871A06CCA314B
:10A9E0001638C2B26748E2749C30FAF7C7FB714868
:10A9F00005706448603000686063A063E063F17CC8
:10AA0000090700E08CE0090F032900D02175A16C33
:10AA1000262917D15949564A8C31C98F1185594B6E
:10AA2000079AB43312881A8788420ADD002808DDA5
:10AA3000002906D0E07D411CE175052802D925706A
:10AA400000E0E575E5700120A073E073A08B5A4922
:10AA5000FF30C33080B2A08388420BD949424018EE
:10AA6000A08338887D21401C80B2C900388088428C
:10AA700000D33D8038887D21C9004843A18B401810
:10AA8000206468E0FFE7FBF70DFF04900898009052
:10AA900004983B6E401CC0B2029A019900F0FCFD84
:10AAA00038490498903103220818427004983039CC
:10AAB00080008446401840687863B86C262806D128
:10AAC00004988C31400041180798008848802D4830
:10AAD0002A4930308C316044898F01802748614693
:10AAE0000B180022796E386E3C46163398540F06C8
:10AAF000000A3843090A521C042AF7DBE16C606B38
:10AB000088421ADA1F4963463031C958002914D0E7
:10AB1000012901D0814210DDE064099806900CE023
:10AB20003A4600210F2003F090FC2079A178401CC8
:10AB3000814202D0002003F09EFB608CE18C8842B1
:10AB400000D2C3E6184A89188842FAD8A07B0128A7
:10AB500001D00221A17303F043FA124A00210F2011
:10AB600003F073FCE07800283BD00A282AD925E0BE
:10AB7000A80000203F420F003C000020280D0020CC
:10AB800041000020800E00208A0000202C080020B8
:10AB90008C0500209A9999999999E13F0000084005
:10ABA000A086010000D02724983A00006800002009
:10ABB0006C00002060000020E7030000E5702570B5
:10ABC000FBF7C6FBFBF78EFAA07C002857D03C4E63
:10ABD0003178617270782072B278E271022917D0F0
:10ABE0004DE0A06BE16C323881420FDAA17920464A
:10ABF000491CC9B2A1710229E4D985710699018461
:10AC0000022101702573FBF7E1FFDBE7A571D9E7AE
:10AC100010280ED02B4F062815D0C8282FD2381850
:10AC2000F11CFAF7ABFA03F0D9FE642003F026F822
:10AC30008AE6254F38684000000E20D1F078FAF7F8
:10AC40007FFD38601BE00222F11CB81DFAF7D5FA2F
:10AC5000002814D0207AE2793818F11CFAF78EFA1D
:10AC600003F0BCFE7D20F988C000FAF741FA1749CD
:10AC700008800146C820FAF73BFA15490880104FB2
:10AC800000269C3F12E00E4975008439785B495BD1
:10AC9000884209D002202070FBF798FF0020207323
:10ACA00007490120B4394853761CF6B22079864210
:10ACB000E9D3084A00210F2003F0C7FB0BB0F0BD19
:10ACC0001C0F0020EC0700207C00002078000020F2
:10ACD0008400002080D027247047000010B504486D
:10ACE000002281898068FCF7FEFCFBF721FF10BD84
:10ACF0009426002010B50448012281898068FCF761
:10AD0000F2FCFBF71BFF10BD94260020C300024895
:10AD1000C15018188280704794260020F0B585B085
:10AD20004848FCF725F84848FDF7D0FB4748FDF7B1
:10AD3000D9FC4748FDF712FF4648FDF70FFF46488C
:10AD4000FDF70CFF00F09EFC14216846FAF72FFA7D
:10AD50000024102611270520029469460007019758
:10AD600000960394FCF7FEFBF5010520029469466A
:10AD70000007019700950394FCF7F4FBFDF778FCBE
:10AD80003648816B0204114381633548016804220F
:10AD90001143016001210846FCF7AAFEFDF78EFB76
:10ADA00000F08AFFFFF702FC002001F03FFF0120C6
:10ADB00001F03CFF022001F039FF0096012605203A
:10ADC00002946946000701960394FCF7CBFB05202B
:10ADD000012210210007FCF786FC05200294694639
:10ADE0000007019600950394FCF7BCFB05200122A7
:10ADF00029460007FCF777FC1A48007800281CD188
:10AE0000194C2068C10718D1184D2968884214D000
:10AE1000174801781748142901D3FF2101E0FF21C9
:10AE200009020160144900680B6814490A68144952
:10AE3000096800F00BFC2068286012A0FEF766FB92
:10AE400005B0F0BD3005002054070020AC070020FD
:10AE5000BC05002044060020CC0600200010024063
:10AE600000700040340000202C000020380000203A
:10AE70003C000020280000201C00002020000020B2
:10AE80002400002077616B752075700D0A000000AA
:10AE9000F0B587B003F03AFD6A4800F097FB6A4EC0
:10AEA000F0806848801C00F091FB30816548001DEF
:10AEB00000F08CFB654D7081FF2001302C466880CE
:10AEC0004034E08C002802D1E1200001E0842179A7
:10AED000717004915E49E88E08705E49E88F0870D1
:10AEE0005D49A88F0870A07930705C49A87A087015
:10AEF0005B48AF8807605B4805210180E8880390C4
:10AF0000FAF7F6F85849088001463846FAF7F0F89B
:10AF10008800081887B2554807807D20C000784314
:10AF2000FAF72AFC524A534BFAF77CFBFAF76AFC11
:10AF3000514980B2088000905048078050480188ED
:10AF4000C820FAF7D5F84F49012208804E4800275B
:10AF500002800398B0807D200499C000002904D1AC
:10AF60003C49B0800A703C490F70B188FAF7C0F8CC
:10AF70004349088045494648009AFCF717FD0028D8
:10AF800001D072B6FEE7A08C012804D0608C414E3F
:10AF9000012838D040E0FF20000203461A4611463F
:10AFA00000F054FBFF25F5352846FCF79DF9FF20FE
:10AFB000000403461A46114600F048FB2846FCF7F9
:10AFC00093F900231A461946184600F03FFB28461D
:10AFD000FCF78AF930486946088072B680212F4D07
:10AFE0002846FBF79DFB002804D00222694628462C
:10AFF000FBF73CFC62B6A78403F0F0FC642002F08F
:10B000003DFE02F05BF867842F8003F0E7FC6420CC
:10B0100002F034FE2248C660208C012807D1278424
:10B0200003F0DCFC642002F029FE1D48C66029887C
:10B030001C48814202D1E888002801D11848C66026
:10B0400007B0F0BD004F000800000020EC07002012
:10B050004002002080000020810000206E000020BF
:10B0600068000020720000207400002070000020A2
:10B07000F853E3A59B843E40760000207A00002030
:10B08000780000208400002082000020FF7F000064
:10B090008C0500200400FA05AAAA0000384A00081E
:10B0A00000ED00E0AA55000000B504494020886288
:10B0B000FF20F53003F0AEFC00BD0000000400509E
:10B0C000FF2302461B0200B519020D489A4202D125
:10B0D00000F0C0F800BD8A4202D100F057F809E044
:10B0E000FF2A04D0824205D100F002F900BD00F031
:10B0F00009F800BD002AFCD100F07AF800BD00007C
:10B10000FFFFFF0000B500F02FF800F02DF800F071
:10B110002BF800F029F800F027F800F025F800F0EF
:10B1200023F800F021F800F01FF800F01DF800F0FF
:10B130001BF800F019F800F017F800F015F800F00F
:10B1400013F800F011F800F0B7F800F0B5F800F0CF
:10B15000B3F800F0B1F800F0AFF800F0ADF800F08F
:10B16000ABF800F0A9F800BD07484021816100BF9D
:10B1700000BF00BF00BF00BF00BF816200BF00BFB3
:10B1800000BF00BF00BF70470004005000B500F0D2
:10B1900093F800F091F800F08FF800F08DF800F0CF
:10B1A0008BF800F089F800F087F800F085F8FFF7D9
:10B1B000DBFFFFF7D9FFFFF7D7FFFFF7D5FFFFF75B
:10B1C000D3FFFFF7D1FFFFF7CFFFFFF7CDFFFFF76B
:10B1D000CBFFFFF7C9FFFFF7C7FFFFF7C5FFFFF77B
:10B1E000C3FFFFF7C1FFFFF7BFFFFFF7BDFF00BDC4
:10B1F00000B5FFF7B9FFFFF7B7FFFFF7B5FFFFF7A0
:10B20000B3FFFFF7B1FFFFF7AFFFFFF7ADFFFFF7AA
:10B21000ABFFFFF7A9FFFFF7A7FFFFF7A5FFFFF7BA
:10B22000A3FFFFF7A1FFFFF79FFFFFF79DFFFFF7CA
:10B230009BFFFFF799FFFFF797FFFFF795FFFFF7DA
:10B2400093FFFFF791FFFFF78FFFFFF78DFFFFF7EA
:10B250008BFF00BD00B5FFF787FFFFF785FFFFF706
:10B2600083FFFFF781FFFFF77FFFFFF77DFFFFF70A
:10B270007BFFFFF779FF00F01FF800F01DF800F0EA
:10B280001BF800F019F800F017F800F015F800F0BE
:10B2900013F800F011F8FFF767FFFFF765FFFFF7FE
:10B2A00063FFFFF761FFFFF75FFFFFF75DFFFFF74A
:10B2B0005BFFFFF759FF00BD0C484021816100BFD3
:10B2C00000BF00BF00BF00BF00BF00BF00BF00BF86
:10B2D00000BF00BF00BF00BF00BF00BF816200BF52
:10B2E00000BF00BF00BF00BF704700000004005057
:10B2F00000B5FFF7E1FFFFF7DFFFFFF7DDFFFFF727
:10B30000DBFFFFF7D9FFFFF7D7FFFFF7D5FFFFF709
:10B31000D3FFFFF7D1FFFFF7CFFFFFF7CDFFFFF719
:10B32000CBFFFFF7C9FFFFF7C7FFFFF7C5FFFFF729
:10B33000C3FFFFF7C1FFFFF7BFFFFFF7BDFFFFF739
:10B34000BBFFFFF7B9FFFFF7B7FFFFF7B5FFFFF749
:10B35000B3FF00BD08B5002808D00246002106480A
:10B360000091044B0068FEF759FA08BD002000F078
:10B3700005F808BD7DB3000824020020044972B618
:10B380000248C860BFF34F8F704700000400FA0501
:10B3900000ED00E0F8B56E4C00256E48E570C18800
:10B3A0007D20C000F9F7A4FE6B4E01463080C82016
:10B3B000F9F79EFE69490880A07A401CA072C00778
:10B3C00006D0E08B411EE183022801D2C820E08331
:10B3D0000A2002F07AFF7D20400102F091FF604FC9
:10B3E0002020BD7278725B48C1887D20C000F9F7CB
:10B3F0007FFE78735B4856490078B8733846203131
:10B4000013380A7802754978417552491E308A7896
:10B410000270C9784170411C4E482030027ECA70CB
:10B42000407E08714B482230027E4A71407E88710E
:10B4300000220C39172003F033F80021172003F005
:10B4400041F8022002F092FF474F01E0FEF74CFD69
:10B4500000210F2002F0A6FE38422063F6D0206BB8
:10B46000411C73D040046FD58122D20100210F20EE
:10B4700002F0EBFF0021102002F094FE4106384854
:10B48000490E0022B430A16402F0DCFE344FB43720
:10B49000787A112858D102223449781DF9F7ADFE87
:10B4A000002851D1F81F027A69460A70407A487024
:10B4B000B97A3180C820F9F71BFE28492C4E088044
:10B4C000387BE08338462838C08E308038462838AC
:10B4D000008FA0832748FCF765FA6084A08B26497B
:10B4E000FF30C33080B2A08388420BD94942401854
:10B4F000A08330882049401C80B20B3130808842C4
:10B5000000D3358030887D21C9004843A18B401885
:10B5100020646846008820841149B87CC7312071B6
:10B52000420008460E469130F9F728FE2079314650
:10B5300042001248F9F722FEE08BFF2804D0257361
:10B5400002202070FBF742FBF8BDFFE701F0C4FDCD
:10B55000A8000020EC0700207800002084000020D4
:10B56000280D00204002002000D027246800002081
:10B570006C0000208C050020E7030000980E0020DE
:10B5800070B586B014216846F9F711FE0E4E002200
:10B5900001213046FCF7A7F801250024009502940C
:10B5A0006946304601950394FBF7DCFF03200190C8
:10B5B00002946946009503943046FBF7D3FF0220BE
:10B5C00002F05CFB06B070BD0004005000887047BC
:10B5D00070470000F8B5044600206A461080194DF7
:10B5E00055222A70AA226A700322AA70661DEE7084
:10B5F0002A716971144A49008918AC712246E81D04
:10B60000F9F7BCFD002007E029186A4689781288FE
:10B6100089186A461180401CB042F5DB611DA81CE8
:10B62000FAF704FE01466846018029190078C871BE
:10B63000684640780872224609320249002001F02B
:10B6400093FBF8BD500C0020EC070020F8B516461F
:10B6500004460F46012205201D46D1030007FCF7D2
:10B6600042F8FFF721FD3846FFF72AFD3046FFF785
:10B6700027FD2846FFF724FD2046FFF721FDFFF7B1
:10B6800013FDF8BD10B5012105200022C9030007F4
:10B69000FCF729F810BD0000FFB5054684001148ED
:10B6A00081B01E46201804220A9FF9F767FD0D4855
:10B6B00004222C3020180399F9F760FD0948094944
:10B6C0005830201806606800B03140183978017091
:10B6D0007978417004480349006D8431085105B000
:10B6E000F0BD0000840F0020A800002010B5FAF77C
:10B6F000B3FCFDF7B1FF00280DD0FDF7ADFF0B2423
:10B70000E40100190069002805D0FDF7A5FF001924
:10B71000016902A08847002010BD00004F4B0D0AB0
:10B720000000000010B5FAF7B5FCFDF795FF002802
:10B730000DD0FDF791FF0B24E401001900690028EA
:10B7400005D0FDF789FF0019016902A08847002094
:10B7500010BD00004F4B0D0A0000000010B502287C
:10B7600014DAFDF779FF00280DD0FDF775FF0B24E3
:10B77000E40100190069002805D0FDF76DFF0019EC
:10B78000016907A088470020C04310BD4868F9F749
:10B7900041FD002801D1FDF7C3FD002010BD0000D0
:10B7A00064656275675F6F666620666C61670D0A27
:10B7B0000000000010B5022814DAFDF74DFF002844
:10B7C0000DD0FDF749FF0B24E401001900690028A2
:10B7D00005D0FDF741FF0019016907A08847002047
:10B7E000C04310BD4868F9F715FD002801D1FDF7E9
:10B7F0009DFD002010BD000064656275675F6F6E7F
:10B8000020666C61670D0A0010B5FFF767FAFDF757
:10B8100023FF00280DD0FDF71FFF0B24E4010019C2
:10B820000069002805D0FDF717FF0019016902A083
:10B830008847002010BD00004F4B0D0A000000009B
:10B8400010B5FFF757FAFDF707FF00280DD0FDF7F9
:10B8500003FF0B24E40100190069002805D0FDF75F
:10B86000FBFE0019016902A08847002010BD0000FE
:10B870004F4B0D0A0000000070B5FDF7EDFE0B25E3
:10B88000ED0100280CD0FDF7E7FE40190069002803
:10B8900006D0FDF7E1FE401902690FA111A0904703
:10B8A000FDF7DAFE002815D0FDF7D6FE4019006935
:10B8B00000280FD0FAF786FBF9F7C2FF04460E46C0
:10B8C000FDF7CAFE401905690B4822460178334648
:10B8D0000AA0A847002070BD76312E302E302E34BD
:10B8E0000000000056657273696F6E3A20202020B8
:10B8F000202025730D0A00003C0000204261747472
:10B900006572793A202020202020257525252025C4
:10B910002E3266560D0A000010B511210248FDF7BF
:10B9200065FE002010BD00006CEA00080020704792
:10B9300010B5072814D0FDF78FFE00280DD0FDF7B5
:10B940008BFE0B24E40100190069002805D0FDF7E7
:10B9500083FE0019016903A088470020C04310BD81
:10B96000002010BD75736167653A207274635F7360
:10B9700065742079797979206D6D20646420686818
:10B98000206D6D2073730D0A0000000010B50020BB
:10B99000FFF7E0FC002010BD10B50B24E4010628E1
:10B9A00012DAFDF759FE00280BD0FDF755FE0019FD
:10B9B0000069002805D0FDF74FFE001901690BA0B2
:10B9C00088470020C04310BDFDF746FE00280BD07D
:10B9D000FDF742FE00190069002805D0FDF73CFE86
:10B9E0000019016911A08847002010BD7365745FBC
:10B9F000616463206E6F726D616C5F6D696E206E45
:10BA00006F726D616C5F6D6178206572726F725FCD
:10BA10006D696E206572726F725F6D6178206572FC
:10BA2000726F725F636E740D0A0000004F4B0D0A57
:10BA30000000000010B50B24E40102280FDAFDF726
:10BA40000BFE00281BD0FDF707FE00190069002837
:10BA500015D0FDF701FE001901690AA00EE0FDF7FF
:10BA6000FBFD00280BD0FDF7F7FD00190069002849
:10BA700005D0FDF7F1FD0019016904A088470020F9
:10BA800010BD00004552524F520D0A004F4B0D0A97
:10BA90000000000070B500250B24ED43E4010228EE
:10BAA0000FDAFDF7D9FD002822D0FDF7D5FD0019EA
:10BAB000006900281CD0FDF7CFFD0019016916A010
:10BAC00015E04868F9F7A6FB002801D0082811D92D
:10BAD000FDF7C2FD00280BD0FDF7BEFD001900697F
:10BAE000002805D0FDF7B8FD001901690EA08847B0
:10BAF000284670BDFDF7B0FD00280BD0FDF7ACFD6A
:10BB000000190069002805D0FDF7A6FD001901699C
:10BB100008A08847002070BD7365745F6465765F18
:10BB200069642069640D0A006964206572726F722D
:10BB30000D0A00004F4B0D0A0000000010B50B2449
:10BB4000E401032812DAFDF787FD00280BD0FDF78A
:10BB500083FD00190069002805D0FDF77DFD00195F
:10BB600001690BA088470020C04310BDFDF774FD9C
:10BB700000280BD0FDF770FD00190069002805D0E2
:10BB8000FDF76AFD001901690AA08847002010BD71
:10BB90007365745F6970205B7365727665725F6947
:10BBA000705D205B7365727665725F706F72745D35
:10BBB0000D0A00004F4B0D0A0000000010B50B24C9
:10BBC000E401032812DAFDF747FD00280BD0FDF74A
:10BBD00043FD00190069002805D0FDF73DFD00195F
:10BBE00001690BA088470020C04310BDFDF734FD5C
:10BBF00000280BD0FDF730FD00190069002805D0A2
:10BC0000FDF72AFD001901690AA08847002010BD30
:10BC10007365745F77696669205B737369645D201F
:10BC20005B70617373776F72645D205B69705D0D2B
:10BC30000A0000004F4B0D0A0000000010B5FFF78E
:10BC40006DF8002010BD10B5FEF74AFB002010BDB6
:10BC5000034A1168382389B2994301431160704740
:10BC60000030014070B5104C2078002811D000251C
:10BC7000012806D002280FD0032801D1FEF770FD5D
:10BC800070BDFFF787FB607B411C617309E0257085
:10BC900070BDFAF75DFB70BDFAF798FF207B411C81
:10BCA00021730528F3D870BDA800002010B5FDF75A
:10BCB000E1FDFBF733FD10BD10B59AB034216846A5
:10BCC000F9F775FA142115A8F9F771FA20210DA8D2
:10BCD000F9F76DFA234801680324E402A143C21472
:10BCE00089180160FBF7FCFE1F48016921430161CF
:10BCF0000E200090FF2001300290102004900220BE
:10BD00000990400401210B900001059100240C9042
:10BD100003910A946846FCF757F9002801D072B6DF
:10BD2000FEE70F2015900320169017941894012118
:10BD3000199415A8FBF7DAFF002801D072B6FEE7C8
:10BD400087200D9003200F94800414901094119478
:10BD50000DA8FBF701FF002801D072B6FEE71AB06C
:10BD600010BD000000700040401002400249014830
:10BD7000886070470050000800ED00E0F0B40268F1
:10BD80000124A407144D154E154FA04205D0A8421A
:10BD900003D0B04201D0B84203D170239A434B681C
:10BDA0001A43A04205D0A84203D0B04201D0B84205
:10BDB00004D103231B029A43CB681A4380239A437E
:10BDC0000B691A4302608A68C262096881620121B4
:10BDD0004161F0BC704700000004004000080140D1
:10BDE0000014014010B4C906C90E01238B40046A37
:10BDF0009C430462036A8A401343036210BC704789
:10BE000030B48468FF252D02AC431B0213430B435F
:10BE10002343836030BC7047826870239A430A438F
:10BE200007210A438260704730B4026A5208520008
:10BE30000262026A446883697025AB439B089B00D9
:10BE40000D681D4302239A438B6813434460856148
:10BE500049684163036230BC704730B4026A102302
:10BE60009A430262036A4568826907242403A24355
:10BE700003242402A2430C68240214432022934387
:10BE80008A6812011A4345608461496881630262CD
:10BE900030BC704730B4026AFF2301339A43026218
:10BEA000026A4468C3697025AB439D08AD000B6806
:10BEB0002B4301256D02AA438D682D021543446072
:10BEC000C3614968C163056230BC704730B4026A1F
:10BED00001231B039A430262036A4568C26907246F
:10BEE0002403A24303242402A2430C682402144323
:10BEF0000122520393438A6812031A434560C461C6
:10BF000049680164026230BC704730B4036A046A55
:10BF10006408640004628469F025AC431201224382
:10BF20000A24A3430B438261036230BC704730B4E0
:10BF3000036A1024A34303628369046A0F252D0357
:10BF4000AB4312031A43A0239C430901214382619E
:10BF5000016230BC7047000070B5FF24114D013400
:10BF6000AC62AF20800001F090FEAC6102F048F9B5
:10BF70000D4C0E4DA06007E002F042F9A060FDF705
:10BF8000B3FF6068401C6060A068A842F4D102F072
:10BF900027F800206060FFF765FE02F021F802F04C
:10BFA00007F870BD00040050880000203001CADE90
:10BFB00010B4818CC90707D001684A6801235B046B
:10BFC0009A43836A1A434A60818C890707D50168BE
:10BFD0004A6801231B049A43C36A1A434A60818C4E
:10BFE000490707D501684A6801239B049A43036BFC
:10BFF0001A434A60818C090707D501684A68012302
:10C00000DB039A43436B1A434A60818CC90607D508
:10C0100001688A6801231B039A43836B1A438A6071
:10C02000818C890607D501688A6801235B039A43DE
:10C03000C36B1A438A60818C490612D501684B682C
:10C0400001221205046C934323434B60016C91421F
:10C0500007D101684A6803235B059A43436C1A437E
:10C060004A60818C090607D501684A680123DB0410
:10C07000806C9A4302434A6010BC7047F0B583B0AD
:10C0800004462646002780367760FBF733FB029094
:10C090002068006825460007603500281CDA2A4819
:10C0A00000900121002249052046029B00F09AFCE5
:10C0B000002811D0EFF31081012080F31088206850
:10C0C000026880239A43026081F310882020E06791
:10C0D0002F76032003B0F0BD20680068400729D503
:10C0E000194800900121002289052046029B00F09A
:10C0F00079FC00281ED0EFF31081012080F3108816
:10C1000020680268FF2321339A43026081F310887C
:10C11000EFF31081012080F31088206882685208B4
:10C120005200826081F31088202030602F76032037
:10C1300003B0F0BD2020E0673060276667662F7689
:10C14000002003B0F0BD0000FFFFFF0110B5806AC2
:10C150000022014640314A834A82FCF721FD10BD8E
:10C16000F8B5846AE06F254680352E6821688968B5
:10C1700000270906002906DA212804D15220075396
:10C18000204600F0DFF820688068400606D5222EA1
:10C1900004D15A200753204600F090F86868102117
:10C1A000084368602046FCF7FBFCF8BD70B501460B
:10C1B000886A0968096800238906002937DB5A2143
:10C1C0000B52EFF31082012181F3108801680C6893
:10C1D000FF250135AC430C6082F31088EFF3108229
:10C1E000012181F3108801688C68640864008C6008
:10C1F00082F31088EFF31082012181F31088016827
:10C200008C684025AC438C6082F31088202280210A
:10C210000A50016E01290AD1EFF3108281F31088D0
:10C2200001680C681025AC430C6082F310884366EB
:10C23000016E012902D0FCF759FF70BD5821095A3F
:10C24000FCF78AFC70BD10B5806A01214166016E61
:10C25000012902D0FCF74EFF10BD5821095A4908A8
:10C26000FCF77AFC10BD10B50146886A09680968B8
:10C2700089061BD4002252210A52EFF310820121B9
:10C2800081F3108801688B688024A3438B6082F35C
:10C290001088EFF31081012282F310880068026891
:10C2A00040231A43026081F3108810BDFDF732F875
:10C2B00010BD10B5806AFDF731F810BD10B4EFF372
:10C2C0001082012181F3108801680B68FF2421345A
:10C2D000A3430B6082F31088EFF31082012181F3F6
:10C2E000108801688B685B085B008B6082F31088A4
:10C2F000016E01290AD1EFF3108281F310880168E1
:10C300000B681024A3430B6082F310882022802145
:10C310000A5000210166816610BC704710B5EFF32A
:10C320001082012181F3108801680B684024A34327
:10C330000B6082F310882021C1670021C166FCF7E1
:10C34000E9FF10BD10B4EFF31082012181F31088D2
:10C3500001680B68C024A3430B6082F3108820217E
:10C36000C16710BC7047000070B5014640318B8B2F
:10C3700002468032156814460268222D04D0906966
:10C3800008210843906170BD526A456D1A402A80A9
:10C39000426D921C42654A8B521E4A834A8B002A88
:10C3A000F1D1EFF31083012282F31088026815683F
:10C3B000FF262136B543156083F31088EFF3108311
:10C3C000012282F31088026895686D086D009560FF
:10C3D00083F3108820222260002484664466184B70
:10C3E00002689A420ED053681B020BD5EFF31083FC
:10C3F000012585F3108815680126B606B54315603A
:10C4000083F31088026E012A02D0FCF76FFE70BD24
:10C410000466EFF31083012282F310880268156826
:10C420001024A543156083F310880268D369DB43A9
:10C43000DB0600D41462098BFCF78EFB70BD000094
:10C440000048004070B5014640318B8B0246803277
:10C45000156814460268222D04D09069082108430B
:10C46000906170BD526A1A40436D1A70426D521C41
:10C4700042654A8B521E4A834A8B002AF1D1EFF360
:10C480001083012282F3108802681568FF26213686
:10C49000B543156083F31088EFF31083012282F314
:10C4A0001088026895686D086D00956083F31088A8
:10C4B00020222260002484664466184B02689A4257
:10C4C0000ED053681B020BD5EFF31083012585F3C3
:10C4D000108815680126B606B543156083F31088E9
:10C4E000026E012A02D0FCF701FE70BD0466EFF374
:10C4F0001083012282F31088026815681024A54376
:10C50000156083F310880268D369DB43DB0600D42F
:10C510001462098BFCF720FB70BD0000004800404E
:10C52000F8B504460025904F20682269A168E369A8
:10C53000114362691A43114302688C4B1A400A4343
:10C54000026020684168032212039143E2681143AC
:10C550004160A0692168B94201D0226A10438A680B
:10C560000B231B029A4302438A6081492268814857
:10C570008A4213D1C0688007800F07D0012809D0F4
:10C58000022805D0032807D0102142E0012140E015
:10C5900002213EE004213CE008213AE076498A424B
:10C5A00013D1C0680C21084007D0042809D00828FE
:10C5B00005D00C2807D010212BE0002129E0022112
:10C5C00027E0042125E0082123E06C498A4201D1BB
:10C5D00000211EE06A498A4201D1002119E0BA42D5
:10C5E00016D1C0680321890208400BD001218902BD
:10C5F000401A0BD0401A07D0884201D1082108E028
:10C60000102106E0002104E0022102E0042100E004
:10C6100010215D485B4E8300BA4236D1002913D009
:10C62000022914D0042917D0082918D00020012588
:10C63000002861D0626851005118814202D811036C
:10C6400081420FD2012589E0FBF754FCF0E7316805
:10C65000C906EDD41846EBE7FBF76CFCE8E70120D0
:10C66000C003E5E7010E06025008002330185941C7
:10C67000F8F754FD03210902444A411A914202D8B5
:10C680002168C8606AE0012568E00122E769D203F9
:10C69000974234D1092919D20F007F443F79FF19FD
:10C6A000BF4404070A140F1414141200FBF722FCF1
:10C6B0000EE0FBF72FFC0BE03168C90608D41846E2
:10C6C00006E0FBF737FC03E0104601E000200125FF
:10C6D000002843D0616840004A088018F8F708FD38
:10C6E00002462B49103A8A4207D8491C01400007EC
:10C6F000420F0A432068C26030E001252EE009297C
:10C7000019D20F007F443F79FF19BF4404070A1470
:10C710000F1414141200FBF7EDFB0EE0FBF7FAFB0D
:10C720000BE03168C90608D4184606E0FBF702FCA6
:10C7300003E0104601E00020012500280ED06168CA
:10C740004A081018F8F7D4FC0146114A10399142F2
:10C7500003D8216880B2C86000E001250020A066EF
:10C76000E0662846F8BD000000480040F369FFEF8E
:10C77000003801404010024000440040004C00409E
:10C78000005000400010024000093D00FFFC0F0077
:10C79000EFFF000070B50446616558200253002188
:10C7A00025468035696022202860606F002819D0F6
:10C7B000214BC362636F21481863636F204858633D
:10C7C000606F81632168666D134624313246606F65
:10C7D000FAF751FD002805D010206860202028605D
:10C7E000012070BD206900280CD0EFF310810120DA
:10C7F00080F3108820680268FF2301331A43026027
:10C8000081F31088EFF31081012080F310882068F5
:10C81000836801221343836081F31088EFF3108152
:10C8200082F310882068826840231A43826081F373
:10C830001088002070BD0000ADC1000847C200088C
:10C8400061C1000870B44165014640310A834A83E2
:10C8500000248466012382681B03FF259A4207D1C6
:10C860000269002A01D08D8319E02B4A8A8316E0E1
:10C870007F26002A09D001252D07AA420ED1026980
:10C88000002A09D03F228A8309E00269002A01D0E8
:10C890008E8304E08D8302E08E8300E08C8301466A
:10C8A00080314C6022220A60EFF31082012181F373
:10C8B000108801688C6801252C438C6082F31088F5
:10C8C0008168994202D10169002912D01349816619
:10C8D0000169002910D0EFF31081012282F3108842
:10C8E00000680268FF2321331A43026081F3108835
:10C8F0000EE00B498166EBE7EFF31081012282F332
:10C9000010880068026820231A43026081F31088AF
:10C9100070BC002070470000FF01000045C4000803
:10C9200069C3000810B4C16F212910D101464031FC
:10C930004A8A002A0DD0C26C03681288D205D20D33
:10C940009A62C26C921CC264488A401E488210BC23
:10C950007047EFF31082012181F3108801680B68A2
:10C960008024A3430B6082F31088EFF3108101222F
:10C9700082F310880068026840231A43026081F342
:10C98000108810BC704710B4C16F21290ED1014628
:10C9900040314A8A002A0BD0C26C036812789A622E
:10C9A000C26C521CC264488A401E488210BC704748
:10C9B000EFF31082012181F3108801680B68802455
:10C9C000A3430B6082F31088EFF31081012282F3FE
:10C9D00010880068026840231A43026081F31088BF
:10C9E00010BC7047FFB583B00C9D04460E46174639
:10C9F0002068C1693046884327D00020B84245D11D
:10CA000020468030029020380190681C36D0FAF71A
:10CA100071FE0699401AA84219D8002D17D0206837
:10CA2000016849072AD5C169C943090712D420689A
:10CA3000082505622046FFF741FC029845600199F0
:10CA400000200876012007B0F0BD0120D6E70320C2
:10CA500007B0F0BDC069C04300050FD401202168B4
:10CA6000C00208622046FFF729FC0298202141609D
:10CA7000019900200876032007B0F0BD2068C16945
:10CA80003046884305D00020B842BED0002007B011
:10CA9000F0BD0120F8E7000010B50248FCF784F86B
:10CAA00010BD00004406002010B50248FCF77CF8D9
:10CAB00010BD0000CC060020F8B51D4D0E0034D08E
:10CAC000032832D2742148431A494418A078002818
:10CAD00002D0012822D028E0E168A06842186068EE
:10CAE0000090406F006840682769101A0818C01B42
:10CAF000F8F7FEFA012905D817D100980068C06937
:10CB0000800612D43878307061692069884201D17A
:10CB1000A06800E0401C2061002506E02046183097
:10CB20003146FCF749FC0028F6D02846F8BD000045
:10CB3000FFFFFFFFBC2B002070B50C00064601D0A4
:10CB4000032E02D30020C04370BD74214843214905
:10CB50000E54227845186A706078A8706068A860E2
:10CB6000A168E9606278002A02D0012A05D00BE0B2
:10CB700028614018401E686106E0284618300123ED
:10CB8000A2686168FCF7F3FBE068E862206928634B
:10CB9000A0692867606968632078002801D00128AF
:10CBA00006D121460C310EC928463830FDF771F800
:10CBB0006078002804D0012806D0022804D006E0BE
:10CBC000304600F009F802E0304600F021F800207D
:10CBD00070BD0000BC2B002038B50C4974225043B6
:10CBE00042185068016804E04C6A6B461C801C883F
:10CBF0001C80CB691B07F7D491681161D368CC18EE
:10CC0000641E54619AB2FCF709FA38BDBC2B0020AF
:10CC100074214843044910B5401801466831406802
:10CC20000122FCF72FFA10BDBC2B002070B5054681
:10CC300074201A4968434418A078002802D00128BB
:10CC400007D00DE0A0682061E1684018401E6061D7
:10CC500006E0204618300123E268A168FCF787FB54
:10CC60006078002801D0012806D121462C310EC958
:10CC700020463830FDF70DF8A078002804D00128B0
:10CC800006D0022804D006E02846FFF7A5FF02E000
:10CC90002846FFF7BDFF002070BD0000BC2B002020
:10CCA00070B50D0001D0032802D30020C04370BD31
:10CCB000742148430449441874212046FCF70AFEB5
:10CCC0000020656070BD0000BC2B002010B502463E
:10CCD0000E490020742343435B185B6893420FD1D5
:10CCE0007422424351188978002906D0012901D0C5
:10CCF000022901D1FFF78CFF10BDFFF76DFF10BDBA
:10CD0000401CC0B20328E5D310BD0000BC2B00209E
:10CD100038B5014613480024742262431218526841
:10CD20008A4219D1742161430818817801290BD0F6
:10CD3000022908D1016F002902D0806EC0B2884755
:10CD40002046FFF765FF38BD816E6A46117069465F
:10CD50001830FCF7F1FAF3E7641CE4B2032CDBD3E0
:10CD600038BD0000BC2B0020F7B582B00021009137
:10CD700003991546002903D0002D01D0032803D3C1
:10CD80000020C04305B0F0BD742148432B4946182C
:10CD9000707834463834002804D0012820D0022886
:10CDA00042D049E0FCF7ECFB20462946FCF743FF64
:10CDB000070033D020463946FCF709FF2A46386879
:10CDC0000399F8F7DBF92046FCF717FF0446FCF758
:10CDD00065FDA088216882B27068FCF7FDF92BE040
:10CDE000FCF7CEFB20462946FCF725FF070015D0AF
:10CDF00020463946FCF7EBFE2A4638680399F8F7D7
:10CE0000BDF92046FCF7F9FE0446FCF747FDA08873
:10CE1000216882B27068FCF739FA0DE0FCF73EFD3C
:10CE20000020C043009007E0134664204343AAB2A9
:10CE300070680399FCF75FF90098A3E7BC2B00200A
:10CE400070B51F4A002174234B439B185B688342D3
:10CE500031D1742041438C186078002816D0012805
:10CE600013D1204638300546FCF7C7FE0146284658
:10CE7000FCF797FE2846FCF7C0FE002805D0818805
:10CE80008AB201686068FCF701FA70BD204638304C
:10CE90000546FCF7B2FE01462846FCF782FE28460E
:10CEA000FCF7ABFE0028F0D081888AB20168606888
:10CEB000FCF792F970BD491CC9B20329C3D370BDF8
:10CEC000BC2B0020F8B53E4C002321783D4A1D467E
:10CED000082910D0072947D0062950D0052952D05B
:10CEE000042953D0032954D0002956D0012958D001
:10CEF00002295AD05BE0A17800264A1F04E0314F96
:10CF0000BF5DFB189BB2761C9642F8DB66792779E9
:10CF10009A195118E3786278C9188918C919401804
:10CF2000C0430006000E1AD1012E14D0022E16D1D5
:10CF300025482449C018F8F721F901F04FFD642075
:10CF400000F09CFEBFF34F8F21492048C860BFF31B
:10CF50004F8F00BFFDE759081046FEF73BFB2570D9
:10CF6000E570A570A571F8BDA1795054491CC8B2EF
:10CF7000A071A178491F8842F5D1082001E06070B6
:10CF800007202070F8BDE0700620FAE760710520E8
:10CF9000F7E7A070E5700420F3E7552807D10120DA
:10CFA000EFE7AA2803D10220EBE7032803D025707E
:10CFB000E570A570F8BD032020702071F8BD000059
:10CFC0009F000020EC0B0020EC0700200400FA0575
:10CFD00000ED00E070B50D48FAF7E4FC0C4C0125BB
:10CFE0002082AD0309E00948FAF7DCFC80B2208218
:10CFF000A189FF392D39884206DBA18980B2884298
:10D00000F1D349198842EED870BD00008C0500208C
:10D01000300100207CB51546024600201C46002940
:10D020000BD0491E00920191044B6A4621462846C6
:10D0300000F0FEF9009A002111707CBD69DB000848
:10D040002021020C01D010211046020A01D0104606
:10D050000839020901D01046091F820801D0104684
:10D06000891E420801D0881E7047081A7047F0B424
:10D07000040C8BB2264682B25E430D0C1046370C70
:10D080005843360480190021794116466E43370C07
:10D0900036048019794126466E438919F0BC7047E1
:10D0A00030B47446641E2578641CAB4200D21D4621
:10D0B000635D5B00E31830BC18470000BFF34F8F7F
:10D0C00004490348C860BFF34F8F00BFFDE700006D
:10D0D0000400FA0500ED00E0BFF34F8F0449034858
:10D0E000C860BFF34F8F00BFFDE700000400FA05E2
:10D0F00000ED00E0004870472C05002002E008C861
:10D10000121F08C1002AFAD170477047002001E0C1
:10D1100001C1121F002AFBD1704708B500216846E3
:10D1200001706B46012202212C2001F09DF90221A1
:10D13000684601706B4601222C2001F095F908BD6C
:10D1400038B504466D20694608706B4601220749D0
:10D150002E2001F089F90649002C01D0054A00E093
:10D16000054A2E2001F066F938BD000006080000CF
:10D1700006180000070600000716000010B5002082
:10D1800000F006F800220421362001F053F910BD0A
:10D1900038B504466B4602220021362001F036F8ED
:10D1A000B3212300FFF77CFF0E0F08153A3A3A3AF5
:10D1B0001C273A3A2F34483A0021684601704078DB
:10D1C0004108490014E06946087880088000401C46
:10D1D00004E06946087880088000801C08701DE023
:10D1E000684602780A404832027041788020014344
:10D1F0006846417012E0684602780A400270407842
:10D200004106490EF4E7694648780221084303E0E5
:10D2100069464878FD210840694648706B460122FE
:10D220000021362001F020F9012200AB1146362002
:10D23000013301F019F938BD69460878CF2108405B
:10D2400069462030CAE708B50321684641700121CC
:10D2500001706B4602220021362001F005F90122FF
:10D26000D20306212D2001F0E5F8012000F006FD93
:10D270000120FFF78DFF08BD08B5020A69464A7014
:10D2800008706B46022204212D2001F0EDF80320E6
:10D29000694608706B46012206212D2001F0E4F852
:10D2A0000020694608706B46012206212D2001F0FE
:10D2B000DBF80A212D2000F075FF08BDF0B51FB482
:10D2C00086B00998089A030D0021024314D05148F2
:10D2D000514A1818504305141198012810981AD073
:10D2E000281A401C00264D4F4D490096019104908C
:10D2F000002812DA444211E01198012449A30128C0
:10D3000001D11098C1430698119A84600360C260ED
:10D3100041600BB0F0BD4042E4E704462105002027
:10D320003F4A001C51410391029012E0E00707D0F0
:10D3300032463B4601990098F8F70CF901910090AC
:10D3400032463B4610461946F8F704F906460F46A2
:10D350006410002CEAD10498039B0028029A0999D2
:10D36000089806DAF8F7F6F8019B009AF8F7F2F851
:10D3700005E0F8F757F9019B009AF8F753F90446CE
:10D380000E460022284BF8F783FA03D80020C0434A
:10D39000014607E00022254B20463146F8F728F8E1
:10D3A000F8F7B2FB102409E0002C0ADB0A22002364
:10D3B000F7F7B4FE079B30321A55641E02460A4343
:10D3C000F2D11122641C079B121B1C19119B012B0B
:10D3D00003D0012308430ED10AE0084304D01120F2
:10D3E00010900020119077E71098151A6D1E0BE031
:10D3F0001098824202DD00236D1C03E0824201DAB4
:10D4000000236D1E002BEED0069811998260C1603A
:10D4100030C07EE701FCFFFF104D0000000014400B
:10D420000000F03F300000000000F0430000E03F4B
:10D43000FFB597B00646002518E2252877D10024CD
:10D440002746FD49049400E00443761C327801200D
:10D45000203A90400842F7D130782A280ED0022294
:10D46000307801463039092916D804990A235943DE
:10D47000303940181443761C0490F1E7189802C81C
:10D4800004911890002904DA012040030443484223
:10D49000049002200443761C30782E2814D10420F6
:10D4A00004437078761C2A2809D11898761C80C805
:10D4B000189009E00A214F43303FC719761C307895
:10D4C000014630390929F5D930786C2810D006DCAE
:10D4D0004C281AD068280ED06A2817D104E0742886
:10D4E00013D07A2812D110E00120400504430CE04B
:10D4F0000121090501E0032109050C4371788142EE
:10D5000003D1012000052418761C761C3078119078
:10D5100066280BD013DC58287DD009DC00287BD08E
:10D520004528F6D04628F4D047281AD1A5E118E0BE
:10D53000632835D0642870D0652812D19DE1702809
:10D540006CD008DC6728F1D069287BD06E280DD01C
:10D550006F2806D1BAE073282ED0752871D07828AC
:10D5600059D01A9A199990476D1C7EE16002400FBC
:10D57000022809D003280DD00428189801680DD07E
:10D580000D60001D189070E11898EA1701680D6091
:10D590004A60F6E7189801680D80F2E70D70F0E731
:10D5A00018986A4601781172001D18900020507278
:10D5B00002A80090012005E0189802C818900020E9
:10D5C0000091C04361070DD5002101E00199491C7C
:10D5D0000191B94212DA8142F8DB009A515C0029CC
:10D5E000F4D10BE0002101E00199491C0191814235
:10D5F000FADB019A0099895C0029F5D10199049818
:10D600001A9B471A21463846199A00F097FA019951
:10D61000401945180BE04FE02CE113E04EE0009874
:10D6200000990078491C00911A9A1999904701981D
:10D63000401E0190401CF2D1214638461A9B199A8F
:10D6400010E137E00A200021009001916002410FB3
:10D65000022907D0189A01CA1892C21794460329C2
:10D6600008D00AE01898C01DC108C90005C9189162
:10D67000944607E000B2C2179446042902D140B292
:10D68000C1178C4600226146944506DA0A460021FD
:10D69000404291418C462D2102E0210504D52B21E9
:10D6A0006A461173012103E0E10701D02021F7E769
:10D6B000029155E00A200AE0102008E010200090B6
:10D6C0000021042004430191082703E008200021E1
:10D6D000019100906002410F022907D0189A01CAF7
:10D6E000189200229446032908D008E01898C01D1B
:10D6F000C108C90005C91891944603E080B2042905
:10D7000000D1C0B200210291210729D511997029B9
:10D7100006D0009A1021019B4A401A4305D00EE022
:10D7200040216A461173012108E06146014306D099
:10D7300030216A4611731199517302210291009AA6
:10D740000821019B4A401A430AD16146014301D195
:10D75000610705D530216A46117301217F1E0291B0
:10D760001199582904D035A10E910DA90D910DE004
:10D7700037A1F9E76146019B009AF7F7CFFC0E9BB2
:10D780008C469B5C0D9A521E0D92137061460143AC
:10D79000F0D10D9805A9081A20300190600703D533
:10D7A00001200004844300E001270198874201DD45
:10D7B000381A00E0002001990090411802980918D9
:10D7C0000498401A0490E00306D421461A9B199A43
:10D7D000049800F0B3F94519002706E003A81A9A47
:10D7E000C05D199990476D1C7F1C02988742F5DB3C
:10D7F000E0030CD521461A9B199A049800F09EF973
:10D80000451904E01A9A3020199990476D1C009927
:10D81000481E00900029F5DC08E00D980D9900786D
:10D82000491C0D911A9A199990476D1C0199481E2F
:10D8300001900029F1DC63E1092801003031323325
:10D84000343536373839616263646566000000003C
:10D850003031323334353637383941424344454626
:10D860000000000000F05AF94519761C30780028B5
:10D8700000D0E2E528461BB0F0BD600700D40627C3
:10D880001898C01DC108C90048680A680831C30F4C
:10D89000DB071891190001D09CA108E0210501D5F2
:10D8A0009BA104E0E10701D09AA100E09AA1430006
:10D8B00011985B08109165280CD006DC452809D02A
:10D8C00046281DD0472841D141E0662818D0672856
:10D8D0003CD13CE00021112F01DB112000E0781C3D
:10D8E0000191009008A911A8FFF7E8FC1399059190
:10D8F0000021119A15927F1C12980197009150E017
:10D900000120C00703900120019008A9009711A8E9
:10D91000FFF7D4FC139A149905920022119B0092F0
:10D9200012981593059A0192002901D0104602E041
:10D93000791C40180190381A01D5019804E0404242
:10D94000401E0090781C0190C01B029043E0012F04
:10D9500000DA01270021112F01DD112000E03846F7
:10D960000191009008A911A8FFF7A8FC139905914F
:10D97000119A0021129815920091019721070CD459
:10D980000599B94201DB019900E00191012904DD0B
:10D99000159A491E515C302906D0B84201DA011DA2
:10D9A00005DA0121029115E00199491EEDE70028F1
:10D9B00005DC0099411800910199091A03E0019AC8
:10D9C000411C914200DD01910099401A401C0290D7
:10D9D0000120C0070390200706D4029901988142D4
:10D9E00002DB0020C043029000206946C87707AFE1
:10D9F000012103980337C907884224D002201190DF
:10DA00002B201290039800280CDA404203902D201E
:10DA1000129007E00A210398F7F76AFB30317F1E66
:10DA2000039039701199481E11900029F2DC039877
:10DA30000028EFD1791E1298087030782021084014
:10DA40004530BF1E387006A8C01BC01D039010983B
:10DA50000078002800D00120019941180298C017D1
:10DA60000918039809180498401A401E0490E0030E
:10DA700006D421461A9B199A049800F05FF84519BC
:10DA800010980078002803D01A9A199990476D1CB5
:10DA9000E00324D521461A9B199A049800F04EF809
:10DAA00045191CE00098002807DB0099059888427A
:10DAB00003DD1598405C199901E0199930201A9AF4
:10DAC000904700986D1C401C00900298401E0290E8
:10DAD000002804D11A9A2E20199990476D1C01999B
:10DAE000481E01900029DDDC05E038781A9A7F1C79
:10DAF000199990476D1C0399481E03900029F4DC86
:10DB000021461A9B199A0498ACE600002D000000EB
:10DB10002B0000002000000000000000F8B50446C3
:10DB200000251E461746880404D405E03946202007
:10DB3000B0476D1C641EF9D52846F8BDFFB50446F4
:10DB4000002581B01E46C80301D5302700E02027FC
:10DB5000880404D505E038460399B0476D1C641E5F
:10DB6000F9D5284605B0F0BD4A68002A06D00A68F3
:10DB7000531C0B6010704868401E486070470000DE
:10DB8000F8B54A002B4B520DD6182B4A0C460546C9
:10DB9000142E2BDA002E12DA284BF7F729FC00227C
:10DBA0001346F7F775FE40D2002C03DA0124E40790
:10DBB00000253AE02046284337D0214C14E0214F7D
:10DBC0000B46F7403B402B4331D01C4BF7F710FC82
:10DBD00000221346F7F75CFE27D2002C03DD01205C
:10DBE0000005F0400419BC4300251EE0332E1EDC66
:10DBF00033460027143BFF43DF40384217D00F4B1A
:10DC0000F7F7A0FC00221346F7F742FE0DD2002CD6
:10DC10000ADD142E0CD03420811B012088404019CD
:10DC2000A84200D2641C0546BD4321462846F8BDE3
:10DC3000641CF9E701FCFFFF9C7500883CE4377E1B
:10DC40000000F03FFFFF0F0010B5FBF799FDFCF758
:10DC50004BF9F8F75DFFFCF7DDFAFCF793FB06489C
:10DC600081880068F9F738FD012802D0F8F712FA28
:10DC700010BDF8F7F1F910BD500000207D2110B55E
:10DC8000C900484300F001F810BD002140E000BF8A
:10DC900000BF00BF00BF00BF00BF00BF00BF00BF8C
:10DCA00000BF00BF00BF00BF00BF00BF00BF00BF7C
:10DCB00000BF00BF00BF00BF00BF00BF00BF00BF6C
:10DCC00000BF00BF00BF00BF00BF00BF00BF00BF5C
:10DCD00000BF00BF00BF00BF00BF00BF00BF00BF4C
:10DCE00000BF00BF00BF00BF00BF00BF00BF00BF3C
:10DCF00000BF00BF00BF00BF00BF00BF00BF00BF2C
:10DD000000BF00BF00BF00BF00BF00BF00BF491C75
:10DD10008142BCD37047000038B50446FFF72EFAA5
:10DD2000FF2252030021282000F08FFB0E4A002121
:10DD3000282000F08AFB0220FFF72AFA0D20FFF7C7
:10DD400027FA042C00D20424224600210A2000F0E5
:10DD50007CFB1020694608706B46012224212F208D
:10DD600000F082FB38BD000000FF5F00FEB50446F6
:10DD70000020064601906079764940000F5A61788C
:10DD800075482578491E6A4601631170042D7CD0C0
:10DD9000072D7AD000210291217801736E49E37931
:10DDA000012292058969002B71D0914381616A48F3
:10DDB000217A4173217A82698907890B0A4382613A
:10DDC0000021042000F041FB3A4664492E2000F077
:10DDD00031FB68460078FFF7B3F9614F0522785DA3
:10DDE000810040185F49431807212B2000F03CFBBD
:10DDF0005D49029801220B180B21282000F034FB0A
:10DE0000785D5A4980000A580C21282000F01DFB3B
:10DE1000E079574980004018A1794900425A02210F
:10DE2000272000F007FB68460078524940000A5A54
:10DE30000421272000F0FEFAE07900282BD0A078FA
:10DE400004282ED028206946087220220621272087
:10DE500000F0F0FA02AB01222621272000F004FB9B
:10DE600068460078444900014018E178890042582A
:10DE70000821272000F0E9FAA17A601C627A0902E1
:10DE8000114313D016E000E001E0012183E71143C4
:10DE9000FF0881618BE764220621272000F0CAFA7F
:10DEA000DEE71020694608720246CFE73349017267
:10DEB000090A4172417A007A0A020243202127208E
:10DEC00000F0B8FA2E4F0C2123203A6800F0BDFA7A
:10DED0006846007804214000C0198288232000F0A1
:10DEE000A9FAA07900280AD0E0792649012243182E
:10DEF0000021212000F0B8FA0320012601902A0712
:10DF0000120F10010243607800218007000B0243CA
:10DF1000019800050243700402432079C0064009BD
:10DF200002436079C00602431F2000F08EFAA078F9
:10DF300061780123084302040748DB030261E179A9
:10DF4000490319430A4302610021082000F07DFAC9
:10DF50000020FEBD4CEB0008182D00200428000016
:10DF6000F4EA00084C0200206A020020FCEA0008E3
:10DF70001CEB000828EB00082CEB00084110000007
:10DF800014EB00086C02002038B50C4607498A8B58
:10DF9000002102432C2000F04DFA684604706B46C5
:10DFA000012206212C2000F05FFA38BD182D002038
:10DFB00010B5FFF7B2F810BD10B5044604213620A5
:10DFC00000F0F0F80121C902002C01D0084300E064
:10DFD000884302460421362000F037FA10BD0000C5
:10DFE00038B540206946087000210E2000F0DAF8AC
:10DFF0000446002211460E2000F027FA6B4601224B
:10E0000000210D2000F030FA074A00210F2000F017
:10E010001CFA00F0F5F9224600210E2000F015FA56
:10E0200002480021017338BDF8FF2724382D002055
:10E03000FEB505460420694608704A4C002060750C
:10E0400021462031206348710873A0836063A06378
:10E0500000F0D6F8444E206002E000F0D1F82060D5
:10E06000B042FAD10020FFF793F800F0C9F8206021
:10E070003E48432101703E4A1F21826041600021D9
:10E080001E2000F0E2F900F0BBF820606B46012290
:10E090000021242000F0E8F91E20FFF7EDF886B2F9
:10E0A000300AA0730420FFF7E7F8074600F0A8F84D
:10E0B00020603806000E0DD002206946087101ABC1
:10E0C000012212212D2000F0CFF9A08B012109039C
:10E0D0000843A08300F094F820600620FFF7CCF8F6
:10E0E00060600720FFF7C8F8A060F006C00E20753A
:10E0F00001D110202075C0B200F0F2F9E80707D076
:10E10000FFF7A1F8A08B0121C9020843A0830AE010
:10E110000521362000F030F8164908400246052156
:10E12000362000F087F90120FFF732F800210420A3
:10E1300000F038F8A0610021262000F033F8152106
:10E140008903084302460021262000F07EF90022C0
:10E150002621362000F06EF900F052F820600020F1
:10E16000FEBD0000182D00203001CADE4002002054
:10E170001F1F1F1FFFFD000038B5094C89B280B278
:10E180006B46022200F042F8002806D1684640782B
:10E19000010268460078081884B2204638BD0000A5
:10E1A000FFFF000038B50024E44389B280B26B461B
:10E1B000042200F02BF8002806D103216846435CB6
:10E1C0002202D418491EFAD5204638BD38B500249D
:10E1D0006B4603222821272000F018F80220694608
:10E1E0000B5C2202D418401EFAD5E00202D5034887
:10E1F000204338BDE002C00A38BD00000000F0FF37
:10E2000010B500210846FFF7CDFF10BD38B5002935
:10E2100009D0402420436C462070C8B27F2906D81C
:10E22000607002200AE069460870012006E0802440
:10E2300020436C466070C809A0700320694600F056
:10E24000A5FB38BD10B5144603460A4621461120E9
:10E25000FFF7DCFF10BD10B5034605220021152095
:10E26000FFF7D4FF10BD10B503460522002117208B
:10E27000FFF7CCFF10BD38B5054600206946087091
:10E2800000F0BEF8FF2401342246002D01D0032205
:10E29000120200210D2000F0CDF8002D13D06B46A6
:10E2A000012203210F20FFF7B1FF68460078000725
:10E2B00009D5FFF795FE224600210D2000F0BAF89F
:10E2C0000020C04338BD002038BD10B504460021F1
:10E2D0001A20FFF767FF000D22030005120B02430F
:10E2E00000211A2000F0B1F810BD000010B5024660
:10E2F00002492E2000F09EF810BD00000418000016
:10E30000F8B505466B46012203210420FFF77EFF86
:10E310000126114C3607002D0DD02A4600210C2075
:10E3200000F088F8694608781021084369460870AB
:10E33000A069304307E069460878EF210840694644
:10E340000870A069B0430B46A0610122032104209C
:10E3500000F08AF8F8BD0000182D002010B5024624
:10E360000021182000F066F810BD0000F8B507463F
:10E37000002568460570B807204C2E4600280ADAAA
:10E380008020694608706B46012200210D2000F0B4
:10E390006BF801202073F8076946087821D0062120
:10E3A0000843694608706B46012200210D2000F0E9
:10E3B0005BF803210F20FFF7DFFE8121C90008422F
:10E3C00019D04020694608706B46012200210D20BB
:10E3D00000F04AF80020FFF7EFFD00252673ED431B
:10E3E00009E002210843694608706B4601220021BA
:10E3F0000D2000F039F82846F8BD0000382D002027
:10E400001CB56B46012203210F20FFF7FFFE684673
:10E4100000784022C1091040C9014000814208D063
:10E42000012069460871024601AB03210D2000F06E
:10E430001BF81CBD08B56B461A70120A5A7089B2D7
:10E4400080B2022200F010F808BD38B500236C46F7
:10E45000E254120A5B1C042BFADB89B280B2234619
:10E46000042200F001F838BD38B58024002909D015
:10E47000C02528436D462870C8B27F2907D8687028
:10E48000022009E0204369460870012004E020438F
:10E490006870C809A8700320694600F0C1FA38BD49
:10E4A00010B51446012312189B029A4202D900208B
:10E4B000C04310BD0B46821E21460920FFF7D4FF42
:10E4C000002010BD10B5054A8905126901430A43B1
:10E4D00000210820FFF7B9FF002010BD182D0020F3
:10E4E00038B504466B4601220E212B20FFF78EFE25
:10E4F00068460078E10640094001C90E01436846BC
:10E5000001706B4601220E212B20FFF7ADFF38BDB5
:10E510007CB5002425466846FFF79DFE0420694629
:10E52000220E2D02154322020C5C1443401EF7D527
:10E53000204629467CBD7CB5002425466846FFF769
:10E5400092FE04206946220E2D02154322020C5C25
:10E550001443401EF7D5204629467CBDF9F7E6F85E
:10E56000FDF7AAFBFBF78EFFFBF754FFFCF72CF837
:10E57000FCF7BCF8FCF7D6F8FCF742F8FCF766F8B5
:10E580004A494B48002522C005608561C56149495B
:10E590000562C1600838F9F795F9002801D072B614
:10E5A000FEE7FCF775FCF8F77BF8F8F749F8FF2071
:10E5B00007214130FFF7E8FCFFF7FAFCF7F77AFC98
:10E5C000F7F732FCFDF75EF8FCF788FBFF2000024E
:10E5D00003461A461146FDF739F8FF24F534204664
:10E5E000F8F782FEFF20000403461A461146FDF7A5
:10E5F0002DF82046F8F778FEFDF744F82E4EB08E41
:10E60000002834D0FCF776FB2C4CB08E002844D088
:10E61000FFF71AFB6169E06A884214D0FF23E361C7
:10E62000226A616AA06AFDF711F8FDF795FCE06ABD
:10E630006061A0892B46401CA081E561226A616A65
:10E64000A06AFDF703F82169E06A8842DDD0206105
:10E650001B480078012823D01AA0FAF757FF224858
:10E6600022490068401E88421CD221A01BE023489A
:10E6700055210170AA214170C3208001FFF74CFB96
:10E6800000221E490D20FFF70BFF00210D20FFF790
:10E6900019FF0020FFF76AFEB6E7F7F74BFEB4E775
:10E6A00017A0DAE71BA0FAF731FFAEE7007C0040C5
:10E6B0008C050020FFFF0000EC0700200000002078
:10E6C00043000020BCD3CBD9B6C8BCC6B4EDCEF352
:10E6D000B4EDCEF3B4EDCEF3A3A1A3A1A3A1A3A166
:10E6E000A3A10D0A00000000DC000020E7030000E9
:10E6F000555742C3BBCECACCE20D0A00400E0020E3
:10E70000BCD3CBD9B6C8BCC6C3BBCECACCE20D0AFB
:10E7100000000000555742B4EDCEF3B4EDCEF3B493
:10E72000EDCEF3A3A1A3A1A3A1A3A1A3A10D0A00D0
:10E7300010B50446FBF770FB4E20FBF73FFBFBF7E1
:10E74000A7FBE0B2FBF73AFBFBF7A2FBFBF764FB8E
:10E750004F20FBF733FBFBF79BFB0020FBF700FB95
:10E760000446FBF775FB204610BD70B50D46044608
:10E77000FBF752FB4E20FBF721FBFBF789FBE0B2D6
:10E78000FBF71CFBFBF784FB2846FBF717FBFBF7AB
:10E790007FFBFBF75DFB0A20FFF777FA70BD0000F7
:10E7A00010B52421002000F04DF81B48FFF76DFA4A
:10E7B00000210F2000F046F80521102000F042F85B
:10E7C0000421112000F03EF883217F2000F03AF868
:10E7D00069217F2000F036F8BD217F2000F032F85B
:10E7E0000E480078262804D1002240218C2000F019
:10E7F00019F8012000F02AF809481421018728207F
:10E8000000F020F80A20FFF740FA012000F036F867
:10E81000012000F043F810BD204E00002802002027
:10E82000EC070020F8B517460E4605460024FFF712
:10E830007FFF3946B44331402143284600F002F8B7
:10E840000020F8BD10B5FFF790FF10BD10B50028EF
:10E850000AD000212720FFF7F5FF04211920FFF738
:10E86000F1FF8721162005E000211620FFF7EAFFBF
:10E8700000211920FFF7E6FF10BD000010B50028A9
:10E8800001D0002200E0802280211120FFF7CAFF82
:10E890000148FFF7FAF910BDA086010010B5002865
:10E8A00011D001212F20FFF7CDFF62213020FFF78B
:10E8B000C9FF46213120FFF7C5FF32210846FFF787
:10E8C000C1FFA22100E022213320FFF7BBFF10BDD2
:10E8D0000C480D4A0188914210D1C18832290DD3CC
:10E8E000C18E43290AD8818F012907D8C08F0128FA
:10E8F00004D8044840308088012801D9012070479D
:10E9000000207047EC070020AA55000010B5012434
:10E91000A40221461948F6F74AFC2246174918482E
:10E92000F7F718FF1548174902888A4224D001805A
:10E93000154981807D21C900C1800A210181002102
:10E94000418181810122C28181834323C3860223C5
:10E950000387E1231B0143878287C2870246403237
:10E96000118451849184C183918014248482118202
:10E97000D384818600F032F810BD0000EC0700203F
:10E9800000FC0008AA55000034120000F0B58C46C7
:10E990000025FF260F4901368E620F4C08E06746BE
:10E9A0007F5DE760A768FF07FCD0E7681F706D1CFC
:10E9B0008542F4DB0020074606E0E760A568ED0726
:10E9C000FCD0E5681D54401C9042F6D38E610020B7
:10E9D000F0BD0000000400500030014070B5FFF7AA
:10E9E00077FF002801D0012070BD72B60124074DC9
:10E9F000A40221462846F7F793FE002804D02246B9
:10EA000003492846F7F732FF62B670BD00FC0008E4
:10EA1000EC070020002100E0491C8142FCD3704734
:10EA2000F0B50025FF260F4F9C4601360B46BE620F
:10EA30000D4C06E0595DE160A168C907FCD0E168B2
:10EA40006D1C8542F6DB002007E06146095CE16051
:10EA5000A168C907FCD0E168401C9042F5D3BE61B3
:10EA60000020F0BD0004005000300140C0EC000860
:10EA700047BC0008A8EC00088DB9000880EC00082D
:10EA800079B8000864EC0008B5B7000838EC000855
:10EA90005DB7000898EC00082DB90008A0EC00084C
:10EAA00031B9000824EC000899B9000890EC00087E
:10EAB0003DBB00082CEC000895BA000858EC000893
:10EAC000BDBB0008B0EC000835BA000878EC0008BF
:10EAD00041B8000850EC000809B8000870EC0008C4
:10EAE00025B7000844EC0008EDB6000888EC0008E3
:10EAF0003DBC00080000010203040005405C00006A
:10EB0000A05C0400C06C0800805C0400E03F1E00B4
:10EB1000E07D1E0007A9022570889B880A00160068
:10EB2000010006000100020087008D002D001A314F
:10EB300052001A339A001A351D011A376B003B3107
:10EB4000BE003B335E013B3596023B3700009959CE
:10EB50009959EB518F421E45142E0080EB51F52838
:10EB60003333E13A703DE13AC235852BC235333358
:10EB7000C235C235AE47E13A5138A33051380000B2
:10EB80000000000000000102030406070809030456
:10EB900006080C10182030000000000102030400D9
:10EBA0004040404040404040404141414141404060
:10EBB0004040404040404040404040404040404055
:10EBC0000502020202020202020202020202020222
:10EBD00020202020202020202020020202020202E9
:10EBE0000290909090909010101010101010101033
:10EBF000101010101010101010101002020202025B
:10EC0000028888888888880808080808080808088A
:10EC10000808080808080808080808020202024054
:10EC2000A0EB00087365745F616463007365745FD3
:10EC30006465765F6964000064656275675F6F662E
:10EC400066000000626565705F6F66660000000028
:10EC50006770735F6F6666007365745F7769666976
:10EC60000000000064656275675F6F6E0000000061
:10EC7000626565705F6F6E006770735F6F6E000036
:10EC8000696E666F00000000736C656570000000BF
:10EC90007365745F697000007274635F6765740008
:10ECA0007274635F736574007265626F6F740000E5
:10ECB0007365745F636F6E7472617374000000003B
:10ECC00074657374000000002B2B2B0D00000000F6
:10ECD00061742B6A6F696E3D6F7461612C31300D08
:10ECE0000000000061742B63683D636E3437302C84
:10ECF000330D000061742B64723D350D000000007F
:10ED000061742B6170706575693D35323639373302
:10ED1000363936653637343834360D0061742B6336
:10ED20006C6173733D610D0061742B6170706B6574
:10ED3000793D32623765313531363238616564325A
:10ED4000613661626637313538383039636634662A
:10ED500033630D0061742B6D6F64653D6D61630DF0
:10ED60000000000061742B6164723D6F66660D00E7
:10ED700061742B7265626F6F740D000061742B7388
:10ED80006C6565703D6C696768742C302C6C6576B9
:10ED9000656C2C6C6F770D0061742B6465766575FE
:10EDA000693D3437333635343966303033312530C8
:10EDB00034780D00636C6561720000006C730000B4
:10EDC000E0ED00080000002030050000385C00087D
:10EDD00080EE000830050020402F00000CD1000814
:10EDE00001534350011204125002368014050214DC
:10EDF0001509090102628139500189072452030C67
:10EE0000E5800CA9B8000C7655AA1122334455664A
:10EE100077889999B213C8EC140854ED1B08D008F0
:10EE20001A1C081A98041119041A28041AF4141A3E
:10EE3000E4041A640C1A7C042A701C310223271380
:10EE40000704380D091E0805400826091040085619
:10EE50000A131D043B08BE0516D8BC401008320139
:10EE6000920402212032021AB48413B1951B08BC0B
:10EE7000084B65969001FF01FF01727201000000CE
:04000005080050C1DE
:00000001FF
